:030000000200AE4D
:03008B00026CC143
:2000AE00127F2C127DC6026CF30820413333395F3620077657616C7465720876773232318C
:2000CE00323939908196E0FCA3E0FDECFAEDFB908192E0D39AA3E064806303809B50030270
:2000EE000103908196E0FAA3E0FBEA908198F0A3EBF0020145908194E0FCA3E0FDECFAEDD2
:20010E00FB908192E0C39AA3E064806303809B4003020135908194E0FAA3E0FBEA90819803
:20012E00F0A3EBF0020145908192E0FAA3E0FBEA908198F0A3EBF0227B00127AAFEA90812C
:20014E00A0F0A3EBF07B00127C059081A0E0FAA3E0FBEA908192F0A3EBF090819AE0FAA349
:20016E00E0FBEA908194F0A3EBF090819CE0FAA3E0FBEA908196F0A3EBF01200D190819809
:20018E00E0FAA3E0FBEA90819EF0A3EBF0227B00126E1C9081A612764F7B00127C0590810C
:2001AE00A612762D9081A212764F22D20E22200E030201C6D2AED2BE2274019081AEF0A335
:2001CE007400F09081AAE0FCA3E0FDECFAEDFB9081AEE0D39AA3E064806303809B4003028F
:2001EE000233C004C0051201BCD005D00474019081ACF0A37400F09081ACE0D3941EA3E0ED
:20020E006480948040030202259081ACE004F07004A3E004F080E09081AEE004F07004A3E6
:20022E00E004F0809E2274019081B0F0A37400F09081B0E0D39405A3E064809480400302A2
:20024E00025E9081B0E004F07004A3E004F080E02274009081B8F09081B7E0FA7B00127C56
:20026E00DEEAC39401FE9081B8E0D39E40030202D69081B8E0FC7D007A007BF6127C13EA83
:20028E00FCEBFD900000EC2582F582E5833DF583C082C0839081B8E0FC7D009081B5E02C3C
:2002AE00FAA3E03DFBEAFCEBFD900000EC2582F582E5833DF583E493D083D082F09081B821
:2002CE00E004F060038090007A007BF6127DBF2274AA905555F07455902AAAF07490905520
:2002EE0055F09081B4E0FC7D009081B2E02CFAA3E03DFBEAFCEBFD900000EC2582F582E5BC
:20030E00833DF583E09081B4F074AA905555F07455902AAAF074F0905555F09081B2E0FC70
:20032E00A3E0FD900000EC2582F582E5833DF583E09081B2F0A3740000F022229081B9E0F0
:20034E005400FAA3E05440FBEA9081B2F0A3EBF09081BBE09081B4F09002DEAA82AB83EAFF
:20036E009081B5F0A3EBF0900349AA82AB839002DEAC02AD03AA82AB83ECC39AFAED9BFB17
:20038E00EA9081B7F012025F9081B4E09081BCF02274AA905555F07455902AAAF074F0905D
:2003AE005555F09081B2E0FCA3E0FD900000EC2582F582E5833DF583E09081B4F022229056
:2003CE0081BDE0FAA3E0FBEA9081B2F0A3EBF090039FAA82AB83EA9081B5F0A3EBF0900321
:2003EE00CCAA82AB8390039FAC02AD03AA82AB83ECC39AFAED9BFBEA9081B7F012025F9074
:20040E0081B4E09081BFF02274AA905555F07455902AAAF074A0905555F09081B2E0FCA3F2
:20042E00E0FD900000EC2582F582E5833DF583C082C0839081B4E0D083D082F09081B2E0B8
:20044E00FCA3E0FD900000EC2582F582E5833DF583E05480FE9081B4E054806E70DE2290C2
:20046E0081C0E0FAA3E0FBEA9081B2F0A3EBF09081C2E09081B4F0900416AA82AB83EA90D4
:20048E0081B5F0A3EBF090046DAA82AB83900416AC02AD03AA82AB83ECC39AFAED9BFBEA3D
:2004AE009081B7F012025F229081C3E0FAA3E0FBEA9081B2F0A3EBF09081C5E09081B4F02F
:2004CE007A007BF6127DBF2274AA905555F07455902AAAF07480905555F074AA905555F0E8
:2004EE007455902AAAF09081B2E0FCA3E0FD900000EC2582F582E5833DF5837430F0908156
:20050E00B2E0FCA3E0FD900000EC2582F582E5833DF583E05480648070E4229081C6E054EF
:20052E0000FAA3E05440FBEA9081B2F0A3EBF09004D6AA82AB83EA9081B5F0A3EBF090050F
:20054E0029AA82AB839004D6AC02AD03AA82AB83ECC39AFAED9BFBEA9081B7F012025F22EB
:20056E009081CCE0D39400A3E0940050030206239081CAE0FAA3E0FBEA9081C0F0A3EBF058
:20058E009081C8E0FCA3E0FD900000EC2582F582E5833DF583E09081C2F012046D74019036
:2005AE0081CEF0A37400F09081CCE0C39401FAA3E09400FB9081CEE0D39AA3E09B40030237
:2005CE0006239081CEE0FCA3E0FD9081CAE02CFAA3E03DFBEA9081C3F0A3EBF09081CEE022
:2005EE00FCA3E0FD9081C8E02CFAA3E03DFBEAFCEBFD900000EC2582F582E5833DF583E072
:20060E009081C5F01204B69081CEE004F07004A3E004F08092229081D4E0D39400A3E09425
:20062E000050030206B774009081D6F0A37400F09081D4E0C39401FAA3E09400FB9081D638
:20064E00E0D39AA3E09B40030206B79081D6E0FCA3E0FD9081D2E02CFAA3E03DFBEAFCEB67
:20066E00FD900000EC2582F582E5833DF583C082C0839081D6E0FCA3E0FD9081D0E02CFA09
:20068E00A3E03DFBEAFCEBFD900000EC2582F582E5833DF583E0D083D082F09081D6E004CC
:2006AE00F07004A3E004F08087229081D8E0FEEE60030206CAC2B2C2B40206D6EE640160C3
:2006CE00030206D9D2B2C2B40206E5EE640260030206E8C2B2D2B40206F4EE6403600302EA
:2006EE0006F7D2B2D2B40206F722904002E0548070F8229081D9E060030207381206F874C2
:20070E0038904000F01206F8740C904000F01206F87402904000F01206F87406904000F0F3
:20072E001206F87401904000F022200A0302073F229081D9E0D39410500302075F1206F8A1
:20074E007401904000F09081D9E0C394109081D9F09081D9E0D3940850030207789081D954
:20076E00E024379081D9F00207839081D9E0C394019081D9F01206F89081D9E04480904060
:20078E0000F074019081E4F09081DAE0FE9081E4E0D39E40030207C81206F89081E4E09069
:2007AE0081DA2582F58250020583E0904001F09081E4E004F0600380CF00229081E5E09034
:2007CE0081D9F09081E67CDA7D8175070A750600127D021207019081F0E0FAA3E0FBEA90F7
:2007EE0081AAF0A3EBF01201C774119081D9F08001009007FF7CDA7D8175070A750600129B
:20080E007D28120701220D6166706E756D206B4D475450459081F212762D12732A9081FED7
:20082E0012764F74079081FCF0A37400F012759D0000803F90820212764F9081FE12762DC2
:20084E0012759D00007A441276716001B340030208D09081FE12762D12759D00007A4412C6
:20086E0076716001B3E433FE9081FCE0C3940DA3E064809480EE82E040030208CD9081FE15
:20088E0012762D12759D00007A441275049081FE12764F90820212762D12759D00007A4497
:2008AE0012748690820212764F9081FCE02401FAA3E03400FBEA9081FCF0A3EBF0809302FB
:2008CE0009769081FE12762D12759D0000803F127671E433FE9081FEC00612762DD006C0B6
:2008EE000612759DEE929321D006C006127671D0066001B3EE82E040030209769081FE12D8
:20090E00762D12759D0000803F127671E433FE9081FCE0D39401A3E064809480B3EE82E062
:20092E0040030209769081FE12762D12759D00007A441274869081FE12764F9082021276B1
:20094E002D12759D00007A4412750490820212764F9081FCE0C39401FAA3E09400FBEA9039
:20096E0081FCF0A3EBF080949081F6E0FCA3E0FD8C828D83C082C0839081FCE090081425A6
:20098E0082F58250020583E493D083D082F090820212762D9081F812764F22C20A740090CF
:2009AE0081D9F08001009009B37CDA7D8175070A750600127D2812070122908046E0648EA2
:2009CE0060030209F474FF90818BF0A3740FF0740090818DF0A37400F0740090818FF0A3E2
:2009EE007410F0020A1274FF90818BF0A37407F0740090818DF0A374F8F0740090818FF045
:200A0E00A37408F07401908206F0908206E0D394084003020B33908206E075F004A490803D
:200A2E00502582F58250020583C082C08312759D00007A4490818BE0FAA3E0FB740112730B
:200A4E0052127660127504908206E075F004A4907FFF2582F5825002058312762D12750478
:200A6E009081F212764F908206E09080942582F58250020583AA82AB83EA9081F6F0A3EB31
:200A8E00F0120822D083D082C082C0839081F812762DD083D08212764F908206E075F00457
:200AAE00A49080702582F58250020583C082C08312759D00007A4490818BE0FAA3E0FB743D
:200ACE0001127352127660127504908206E075F004A490801F2582F5825002058312762DDC
:200AEE001275049081F212764F908206E090809C2582F58250020583AA82AB83EA9081F69C
:200B0E00F0A3EBF0120822D083D082C082C0839081F812762DD083D08212764F908206E0C1
:200B2E0004F0020A1822D295908207E0C39401908207F0908207E0FE7403FAEEC333DAFC8A
:200B4E00908207F0908207E0540864086003020B6B908207E054F74440908207F0908046BB
:200B6E00E0FE908207E04E908207F0D296740190820CF090820CE0D394084003020BBB9046
:200B8E008207E0548024FFB39294120234C295908207E0FE7401FAEEC333DAFC908207F046
:200BAE00120234D29590820CE004F080C6D294908208E0FCA3E0FD8C828D837400F0A374CB
:200BCE0000F090820AE0FCA3E0FD8C828D837400F0A37400F0A291740033FEA2E9EE82E063
:200BEE0050F3C295740190820CF090820CE0D3940C4003020CE1120234D295908208E0FC82
:200C0E00A3E0FD8C828D83C082C083908208E0FCA3E0FD8C828D837C017D00E0FAA3E0FBBD
:200C2E00127CC4EAD083D082F0A3EBF090820AE0FCA3E0FD8C828D83C082C08390820AE040
:200C4E00FCA3E0FD8C828D837C017D00E0FAA3E0FB127CC4EAD083D082F0A3EBF012023403
:200C6E00209003020CA2908208E0FCA3E0FD8C828D83C082C083908208E0FCA3E0FD8C8266
:200C8E008D83E04401FAA3E04400FBEAD083D082F0A3EBF020E803020CD690820AE0FCA3CE
:200CAE00E0FD8C828D83C082C08390820AE0FCA3E0FD8C828D83E04401FAA3E04400FBEA45
:200CCE00D083D082F0A3EBF0C29590820CE004F0020BF8908208E0FCA3E0FD8C828D83C051
:200CEE0082C08390818BE0FCA3E0FDD083D082E0FAA3E0FBD3127D645003020D3A908208B0
:200D0E00E0FCA3E0FD8C828D83C082C083908208E0FCA3E0FD8C828D83E0C39400FAA3E07E
:200D2E009410FBEAD083D082F0A3EBF090820AE0FCA3E0FD8C828D83C082C08390818BE072
:200D4E00FCA3E0FDD083D082E0FAA3E0FBD3127D645003020D9390820AE0FCA3E0FD8C82CB
:200D6E008D83C082C08390820AE0FCA3E0FD8C828D83E0C39400FAA3E09410FBEAD083D0DA
:200D8E0082F0A3EBF0C2962290820D12762D12759D000000001276716003020DE180090806
:200DAE0020302E3030303030900DAD7C1D7D8275070A750600127D28908211E090821DF0FB
:200DCE0090821D7C127D8275070B750600127D02020E5F90820D12762D12759D00002041EE
:200DEE001276714003020E2190820D12762D90821D7E087F05126F0E908211E090821DF0BA
:200E0E0090821D7C127D8275070B750600127D02020E5F90820D12762D90821D7E087F05F9
:200E2E00126F0E908211E0C3940190821DF07420FB7A01127A317802E41279AD90821D749B
:200E4E00011279AD7C127D8275070B750600127D022275B1A0744190F700F0908228E0FEFF
:200E6E00EE6003020E7D747190F704F0020E8BEE64016003020E8E745390F704F0020E9C49
:200E8E00EE64026003020E9F744990F704F0020EADEE64036003020EB0744790F704F00239
:200EAE000EBEEE64046003020EC1744390F704F0020ECFEE64056003020ED2744190F704E1
:200ECE00F0020EE0EE64066003020EE3744090F704F0020EE3742590F705F0740790F7013C
:200EEE00F07400908227F0740190822AF090822AE0D3940F4003020FBF90822AE075F01080
:200F0E00A490F7002582F582500205837455F090822AE075F010A490F7002582F5825002BB
:200F2E000583A37455F090822AE075F010A490F7002582F58250020583A3A3A3A3A3A374C5
:200F4E0000F090822AE075F010A490F7002582F58250020583A3A37400F090822AE075F0B4
:200F6E0010A490F7002582F58250020583A3A3A37400F090822AE075F010A490F700258280
:200F8E00F58250020583A3A3A3A37400F090822AE075F010A490F7002582F582500205834E
:200FAE00A3A3A3A3A37400F090822AE004F0020EFB908229E0FE7401FAEEC333DAFC90F7AC
:200FCE0000F0908229E0540164016003020FEAE59AFEEE4402F59AD2AF020FF3E59AFE742A
:200FEE0002F45EF59A22200F03021005E59AFEEE4402F59A02100EE59AFE7402F45EF59A61
:20100E00227C037D0090822BE0FAA3E0FB127CD1EA90F706F07C057D0090822BE0FAA3E0B1
:20102E00FB127CC4EA90F707F07C037D0090822DE0FAA3E0FB127CD1EA90F70CF090F70DFA
:20104E00E0541F7C057D00FE90822DE0FAA3E0FB127CC4EA4E90F70DF02290823012782A76
:20106E001277AC1500000012775674011277C6EA90F708F090823012782A1277AC0D0000D4
:20108E000012775674011277C6EA90F709F090823012782A1277AC050000001277567401B1
:2010AE001277C6EA90F70AF090823012782A1277AC0300000012776774011277C6EA54F850
:2010CE0090F70BF090823412782A1277AC1500000012775674011277C6EA90F70CF090821A
:2010EE003412782A1277AC0D00000012775674011277C6EA90F70DF090823412782A127724
:20110E00AC0500000012775674011277C6EA90F70EF090823412782A1277AC0300000012BA
:20112E00776774011277C6EA54F890F70FF02290823AE0FEEE6003021161908239E075F0A2
:20114E0010A490F7002582F58250020583747FF0021196EE64016003021199908239E075C0
:20116E00F010A490F7002582F58250020583A374FBF0908239E075F010A490F7002582F5D5
:20118E00825002058374BFF00211CEEE640260030211D1908239E075F010A490F7002582D4
:2011AE00F58250020583A374D7F0908239E075F010A490F7002582F5825002058374BFF00C
:2011CE00021206EE64036003021209908239E075F010A490F7002582F58250020583A37438
:2011EE00E7F0908239E075F010A490F7002582F5825002058374BFF00212092290823BE0B8
:20120E0075F010A490F7002582F58250020583A3A3A3A3A3A3C082C08390823BE075F0102F
:20122E00A490F7002582F58250020583A3A3A3A3A3A3E054F74408D083D082F090823BE072
:20124E00908239F090823CE090823AF012113D2290823DE075F010A490F7002582F582501C
:20126E00020583A3A3A3A3A3A3C082C08390823DE075F010A490F7002582F58250020583B8
:20128E00A3A3A3A3A3A3E054F7D083D082F090823DE0908239F090823EE090823AF01211B5
:2012AE003D2290823FE075F010A490F7002582F58250020583E05482FE90823FE075F0109E
:2012CE00A490F7002582F58250020583A3E0FA7401FCEAC313DCFC54554EFE90823FE075BC
:2012EE00F010A490F7002582F58250020583A3A3A3A3A3A3E054084EFE90823FE075F010BD
:20130E00A490F7002582F58250020583A3A3A3A3A3A3E0FA7403FCEAC333DCFC54204E9073
:20132E008240F022908241E075F010A490F7002582F58250020583A3A37C037D00C082C0BC
:20134E0083908242E0FAA3E0FB127CD1EAD083D082F0908241E075F010A490F7002582F503
:20136E008250020583A3A3A37C057D00C082C083908242E0FAA3E0FB127CC4EA54E0D08328
:20138E00D082F0908241E075F010A490F7002582F58250020583A3A3A3A3A3A3C082C083DB
:2013AE00908241E075F010A490F7002582F58250020583A3A3A3A3A3A3E054FBD083D082AE
:2013CE00F022908244E075F010A490F7002582F58250020583A3A3C082C083908245127873
:2013EE002A1277AC1500000012775674011277C6EAD083D082F0908244E075F010A490F773
:20140E00002582F58250020583A3A3A3C082C08390824512782A1277AC0D0000001277562C
:20142E0074011277C6EAD083D082F0908244E075F010A490F7002582F58250020583A3A347
:20144E00A3A3C082C08390824512782A1277AC0500000012775674011277C6EAD083D0823C
:20146E00F0908244E075F010A490F7002582F58250020583A3A3A3A3A3C082C08390824595
:20148E0012782A1277AC0300000012776774011277C6EA54F8D083D082F0908244E075F038
:2014AE0010A490F7002582F58250020583A3A3A3A3A3A3C082C083908244E075F010A490B5
:2014CE00F7002582F58250020583A3A3A3A3A3A3E054FB4404D083D082F022908249E0755F
:2014EE00F010A490F7002582F58250020583A3A3A3A3A3A3E05404640460030215E59082D8
:20150E0049E075F010A490F7002582F58250020583A3A3E0FA7B00E41277C690824E127844
:20152E004090824E12782A1277AC08000000127767908249E075F010A490F7002582F58223
:20154E0050020583A3A3A3E0FA7B00E41277C612774890824E12784090824E12782A12779A
:20156E00AC08000000127767908249E075F010A490F7002582F58250020583A3A3A3A3E07A
:20158E00FA7B00E41277C612774890824E12784090824E12782A1277AC050000001277675C
:2015AE00908249E075F010A490F7002582F58250020583A3A3A3A3A3E0FE7403FAEEC31308
:2015CE00DAFC541FFA7B00E41277C612774890824E12784002164A908249E075F010A490CB
:2015EE00F7002582F58250020583A3A3E0FA7B00E41277C690824E12784090824E12782AE2
:20160E001277AC03000000127767908249E075F010A490F7002582F58250020583A3A3A3D8
:20162E00E0FE7405FAEEC313DAFC5407FA7B00E41277C612774890824E12784090824E1241
:20164E00782A90824A12784022908253E0D3940850030216697408908253F0908253E0D321
:20166E00940050030216FB908252E075F010A490F7002582F58250020583C082C08374008D
:20168E00908256F0908253E0C39401FE908256E0D39E40030216F7E58124FFF88682088627
:2016AE0083A3A3A3A3A3A3A3C082C083908256E0D083D0822582F58250020583C082C08335
:2016CE00908254E0FCA3E0FD8C828D83E0D083D082F0908254E004F07004A3E004F0908270
:2016EE0056E004F06003809C00D083D082908252E075F010A490F7002582F58250020583B2
:20170E00A3A3A3A3A3A3C082C083908252E075F010A490F7002582F58250020583A3A3A39F
:20172E00A3A3A3E0540FFE908253E0540FC44ED083D082F0908227E0600302179C90F70169
:20174E00E0641824FFE433FE90F701E0641F24FFEE72E0400302177490F701E0908227F038
:20176E00740790F701F0908252E075F010A490F7002582F58250020583A3E05402640260ED
:20178E000302179C908227E04420908227F0908252E075F010A490F7002582F58250020584
:2017AE0083A374FEF022908258E0FCA3E0FD8C828D83C082C083908257E075F010A490F71F
:2017CE00002582F58250020583A3A3A3A3A3A3E0C4540FD083D082F0908258E0FCA3E0FDCF
:2017EE008C828D83E0D39408500302180A908258E0FCA3E0FD8C828D837408F0908258E05D
:20180E00FCA3E0FD8C828D83E0D3940050030218B6908257E075F010A490F7002582F582AF
:20182E0050020583C082C083740090825CF0908258E0FCA3E0FD8C828D83E0C39401FE90BF
:20184E00825CE0D39E40030218B290825AE0FCA3E0FD8C828D83C082C083E58124FDF886CC
:20186E0082088683C082C083D083D082A3A3A3A3A3A3A3C082C08390825CE0D083D082258B
:20188E0082F58250020583E0D083D082F090825AE004F07004A3E004F090825CE004F06025
:2018AE0003808B00D083D082908227E0600302191090F701E0641824FFE433FE90F701E03C
:2018CE00641F24FFEE72E040030218E890F701E0908227F0740790F701F0908257E075F09D
:2018EE0010A490F7002582F58250020583A3E0540864086003021910908227E0442090823F
:20190E0027F0908257E075F010A490F7002582F58250020583A374FDF02290825DE090823A
:20192E003FF01212B0908240E054806480600302195390825DE090823FF01212B090824025
:20194E00E0544170ED90825DE0908239F0740090823AF012113D90825DE0908241F0908269
:20196E005EE0FAA3E0FBEA908242F0A3EBF012133290825DE0908252F0908260E090825346
:20198E00F0908261E0FAA3E0FBEA908254F0A3EBF012165790825DE090823BF0740390822C
:2019AE003CF012120A22908265E075F004A4907FFF2582F5825002058312762D908263E029
:2019CE00FAA3E0FB740112735212766012750412759D00007A4412750490826612764F22E4
:2019EE0090826A12762D90826EE075F004A4907FFF2582F5825002058312762D1274861262
:201A0E00759D00007A44127486127331EA908192F0A3EBF074D0908194F0A3748AF074301D
:201A2E00908196F0A37475F01200D1908198E0FAA3E0FBEA90826FF0A3EBF022908273E041
:201A4E0075F004A490801F2582F5825002058312762D908271E0FAA3E0FB74011273521256
:201A6E00766012750412759D00007A4412750490827412764F2290827812762D90827CE05E
:201A8E0075F004A490801F2582F5825002058312762D12748612759D00007A441274861243
:201AAE007331EA908192F0A3EBF074D0908194F0A3748AF07430908196F0A37475F0120046
:201ACE00D1908198E0FAA3E0FBEA90827DF0A3EBF02230EC03021AEF7401908280F0021AE0
:201AEE00F57400908280F030B303021B05908280E04402908280F030B503021B15908280FF
:201B0E00E04404908280F0908280E090827FF022121AE090827FE0908282F0A209740033A5
:201B2E00FE908282E024FFEE82E04003021B8074019081E5F0800908204C6F636B65642054
:201B4E00901B457CE67D8175070A750600127D2874649081F0F0A37400F01207C9740090B9
:201B6E008281F07400908187F07400908188F0021C3E908188E06003021BA7740090828168
:201B8E00F07400908187F0908282E06003021BA47401908188F0021C3E908282E0FE9081D6
:201BAE0087E06E908283F0908283E07003021C01908188E0C3940A4003021BF27401908104
:201BCE0088F0908283E0FE7404FAEEC333DAFCFE908282E04E908281F0908282E090818791
:201BEE00F0021BFE7400908188F07400908281F0021C3E908188E0C3940AE433FE908282F9
:201C0E00E0D39400B3EE82E04003021C2E908188E02401908188F07400908281F0021C366B
:201C2E00908282E0908281F0908282E0908187F022C2097400908187F07400908188F0229B
:201C4E00908284E0D394085003021C63740190804CF0021C80908284E0C394014003021C2F
:201C6E0078740890804CF0021C80908284E090804CF090804CE0FA7B0090804E7F01E41231
:201C8E006F2322200B03021CCB90804DE0240190804DF090804DE0540464046003021CCB73
:201CAE0074119081D9F0800100901CB67CDA7D8175070A750600127D28120701229080007C
:201CCE00E0FEEE6003021E517420FB7A017802908051127D476003021CF87449FB7A017877
:201CEE0002908051750703127CF490804CE075F002A49080A32582F58250020583E0FAA303
:201D0E00E0FBEA908263F0A3EBF090804CE0908265F01219B490826612762D90804CE075AD
:201D2E00F004A49080502582F5825002058312762D12750490820D12764F7406908211F0E2
:201D4E00120D969082127C857D8275070A750600127D0274019081D9F0127A319080517429
:201D6E00011279AD90828574011279AD90804CE09080942582F58250020583E0FB7A017832
:201D8E0002E41279AD7CDA7D8175070A750600127D0212070190804CE075F002A49080E3DD
:201DAE002582F58250020583E0FAA3E0FBEA908271F0A3EBF090804CE0908273F0121A4AC3
:201DCE0090827412762D90804CE075F004A49080702582F5825002058312762D1275049029
:201DEE00820D12764F7406908211F0120D969082127C857D8275070A750600127D027409FA
:201E0E009081D9F0127A3190804E74011279AD90828574011279AD90804CE090809C25823F
:201E2E00F58250020583E0FB7A017802E41279AD7CDA7D8175070A750600127D0212070157
:201E4E00021FD1EE64026003021FD47420FB7A017802908051127D476003021E7B743EFB70
:201E6E007A017802908051750703127CF490804CE075F002A49080B32582F58250020583FB
:201E8E00E0FAA3E0FBEA908263F0A3EBF090804CE0908265F01219B490826612762D908050
:201EAE004CE075F004A49080502582F5825002058312762D12750490820D12764F74069043
:201ECE008211F0120D969082127C857D8275070A750600127D0274019081D9F0127A31906A
:201EEE00805174011279AD90828574011279AD90804CE09080942582F58250020583E0FB5F
:201F0E007A017802E41279AD7CDA7D8175070A750600127D0212070190804CE075F002A45B
:201F2E009080F32582F58250020583E0FAA3E0FBEA908271F0A3EBF090804CE0908273F0B4
:201F4E00121A4A90827412762D90804CE075F004A49080702582F5825002058312762D123A
:201F6E00750490820D12764F7406908211F0120D969082127C857D8275070A750600127DEE
:201F8E000274099081D9F0127A3190804E74011279AD90828574011279AD90804CE0908082
:201FAE009C2582F58250020583E0FB7A017802E41279AD7CDA7D8175070A750600127D02AD
:201FCE00120701022154EE640160030221577420FB7A017802908051127D476003021FFEF5
:201FEE00743CFB7A017802908051750703127CF490804CE075F002A49080C32582F5825049
:20200E00020583E0FAA3E0FBEA908263F0A3EBF090804CE0908265F01219B4908266127681
:20202E002D90804CE075F004A49080502582F5825002058312762D12750490820D12764F8E
:20204E007406908211F0120D969082127C857D8275070A750600127D0274019081D9F01219
:20206E007A3190805174011279AD90828574011279AD90804CE09080942582F58250020500
:20208E0083E0FB7A017802E41279AD7CDA7D8175070A750600127D0212070190804CE07512
:2020AE00F002A49081032582F58250020583E0FAA3E0FBEA908271F0A3EBF090804CE09071
:2020CE008273F0121A4A90827412762D90804CE075F004A49080702582F582500205831289
:2020EE00762D12750490820D12764F7406908211F0120D969082127C857D8275070A750647
:20210E0000127D0274099081D9F0127A3190804E74011279AD90828574011279AD90804C61
:20212E00E090809C2582F58250020583E0FB7A017802E41279AD7CDA7D8175070A750600CC
:20214E00127D021207010222D7EE640360030222DA7420FB7A017802908051127D476003F7
:20216E00022181744CFB7A017802908051750703127CF490804CE075F002A49080D32582CA
:20218E00F58250020583E0FAA3E0FBEA908263F0A3EBF090804CE0908265F01219B4908227
:2021AE006612762D90804CE075F004A49080502582F5825002058312762D12750490820DF6
:2021CE0012764F7406908211F0120D969082127C857D8275070A750600127D02740190819C
:2021EE00D9F0127A3190805174011279AD90828574011279AD90804CE09080942582F582FB
:20220E0050020583E0FB7A017802E41279AD7CDA7D8175070A750600127D021207019080DA
:20222E004CE075F002A49081132582F58250020583E0FAA3E0FBEA908271F0A3EBF09080FA
:20224E004CE0908273F0121A4A90827412762D90804CE075F004A49080702582F5825002E5
:20226E00058312762D12750490820D12764F7406908211F0120D969082127C857D827507B0
:20228E000A750600127D0274099081D9F0127A3190804E74011279AD90828574011279ADB7
:2022AE0090804CE090809C2582F58250020583E0FB7A017802E41279AD7CDA7D8175070A6A
:2022CE00750600127D0212070102239AEE6404600302239D7420FB7A017802908051127D1C
:2022EE004760030223047457FB7A017802908051750703127CF490804CE075F002A4908188
:20230E00632582F58250020583E0FAA3E0FB9082857F077401126F2374019081D9F0127AEB
:20232E003190805174011279AD90828574011279AD7CDA7D8175070A750600127D0212070D
:20234E000190804CE075F002A49081732582F58250020583E0FAA3E0FB9082857F077401C1
:20236E00126F2374099081D9F0127A3190804E74011279AD90828574011279AD7CDA7D81F4
:20238E0075070A750600127D0212070102239D200C030223B67421FB7A017802908051755C
:2023AE000703127CF40223C67420FB7A017802908051750703127CF422740190828FF090FA
:2023CE00828FE0D39408400302248290828FE075F002A49080B32582F58250020583C0821B
:2023EE00C08390818BE0FAA3E0FBEAD083D082F0A3EBF090828FE075F002A49080C3258295
:20240E00F58250020583C082C08390818DE0FAA3E0FBEAD083D082F0A3EBF090828FE075EF
:20242E00F002A49080F32582F58250020583C082C08390818BE0FAA3E0FBEAD083D082F005
:20244E00A3EBF090828FE075F002A49081032582F58250020583C082C08390818DE0FAA3B8
:20246E00E0FBEAD083D082F0A3EBF090828FE004F00223CD227C057D00908290E0FAA3E0F0
:20248E00FB127CD1EA908292F0227C057D00908293E0FAA3E0FB127CC4908043E0FCA3E035
:2024AE00FDEA4CFAEB4DFBEA908295F0A3EBF02290829712762D90829F12764F9082A2E013
:2024CE009082A3F09082A1E09082A4F09082A0E09082A5F090829FE09082A6F09082A312D7
:2024EE00762D90829B12764F229082ABE09082B3F09082ACE09082B4F09082ADE09082B579
:20250E00F09082AEE09082B6F09082AFE09082B7F09082B0E09082B8F09082B1E09082B941
:20252E00F09082B2E09082BAF09082A7E090825DF09082A8E0FAA3E0FBEA908293F0A3EB26
:20254E00F0122498908295E0FAA3E0FBEA90825EF0A3EBF09082AAE0908260F09082B3AA7B
:20256E0082AB83EA908261F0A3EBF0121928229082BEE09082C4F09082BFE09082C5F090DF
:20258E0082C012762D90829712764F1224BE90829B12762D9082C612764F9082BBE09082F2
:2025AE005DF09082BCE0FAA3E0FBEA908293F0A3EBF0122498908295E0FAA3E0FBEA9082D4
:2025CE005EF0A3EBF07406908260F09082C4AA82AB83EA908261F0A3EBF0121928229082C3
:2025EE00CAE0FCA3E0FD8C828D83E0600302261F9082CAE0FCA3E0FD8C828D837401F090B4
:20260E0082CCE0FCA3E0FD8C828D837408F00226419082CCE0FCA3E0FD8C828D83C082C0B5
:20262E00839082CAE0FCA3E0FD8C828D83E0D083D082F022C20F120FF49082D0E0FCA3E0F5
:20264E00FD8C828D83C082C0839082CEE0FCA3E0FD8C828D83E0FAA3E0FBEAD083D082F09B
:20266E00A3EBF0D20F120FF42274D39082CAF0A37482F074D59082CCF0A37482F01225EC57
:20268E009082D2E024FFB3E433FE9082D2E0640124FFB3EE72E040030227419082D3E0903C
:2026AE0082D4F09082D5E0FE9082D4E0D39E400302274174019082A7F074039082A8F0A33B
:2026CE007400F074049082AAF074019082ABF09082D4E09082ACF09082D4E075F002A4906D
:2026EE0081632582F58250020583E0FAA3E0FBEB9082ADF09082D4E075F002A49081632594
:20270E0082F58250020583E09082AEF074009082AFF074009082B0F074009082B1F0740062
:20272E009082B2F01224F79082D4E004F060030226B1009082D2E024FFB3E433FE9082D221
:20274E00E0640224FFB3EE72E040030227F49082D3E09082D4F09082D5E0FE9082D4E0D3B6
:20276E009E40030227F474019082A7F074039082A8F0A37400F074049082AAF0740290825B
:20278E00ABF09082D4E09082ACF09082D4E075F002A49081732582F58250020583E0FAA352
:2027AE00E0FBEB9082ADF09082D4E075F002A49081732582F58250020583E09082AEF07445
:2027CE00009082AFF074009082B0F074009082B1F074009082B2F01224F79082D4E004F0DE
:2027EE006003022764002274D79082CAF0A37482F074D99082CCF0A37482F01225EC908240
:20280E00D6E024FFB3E433FE9082D6E0640124FFB3EE72E040030228A29082D7E09082D804
:20282E00F09082D9E0FE9082D8E0D39E40030228A274019082BBF074089082BCF0A3740004
:20284E00F074019082BEF09082D8E09082BFF09082D8E075F002A49080A32582F5825002C2
:20286E000583E0FAA3E0FBEA908263F0A3EBF09082D8E0908265F01219B490826612762D60
:20288E009082C012764F12257D9082D8E004F06003808E009082D6E024FFB3E433FE9082D9
:2028AE00D6E0640224FFB3EE72E040030229389082D7E09082D8F09082D9E0FE9082D8E0FC
:2028CE00D39E400302293874019082BBF074089082BCF0A37400F074029082BEF09082D840
:2028EE00E09082BFF09082D8E075F002A49080E32582F58250020583E0FAA3E0FBEA908215
:20290E0071F0A3EBF09082D8E0908273F0121A4A90827412762D9082C012764F12257D90ED
:20292E0082D8E004F06003808E002274DB9082CAF0A37482F074DD9082CCF0A37482F0126A
:20294E0025EC9082DAE024FFB3E433FE9082DAE0640124FFB3EE72E04003022A039082DBFB
:20296E00E09082DCF09082DDE0FE9082DCE0D39E4003022A0374019082A7F0740A9082A8B7
:20298E00F0A37400F074049082AAF074019082ABF09082DCE09082ACF09082DCE075F0023B
:2029AE00A49080A32582F58250020583E0FAA3E0FBEB9082ADF09082DCE075F002A49080DF
:2029CE00A32582F58250020583E09082AEF074009082AFF074009082B0F074009082B1F04C
:2029EE0074009082B2F01224F79082DCE004F06003022973009082DAE024FFB3E433FE906A
:202A0E0082DAE0640224FFB3EE72E04003022AB69082DBE09082DCF09082DDE0FE9082DC65
:202A2E00E0D39E4003022AB674019082A7F0740A9082A8F0A37400F074049082AAF074022B
:202A4E009082ABF09082DCE09082ACF09082DCE075F002A49080E32582F58250020583E09B
:202A6E00FAA3E0FBEB9082ADF09082DCE075F002A49080E32582F58250020583E09082AED2
:202A8E00F074009082AFF074009082B0F074009082B1F074009082B2F01224F79082DCE0A3
:202AAE0004F06003022A26002274DF9082CAF0A37482F074E19082CCF0A37482F01225ECC6
:202ACE009082DEE024FFB3E433FE9082DEE0640124FFB3EE72E04003022B649082DFE090AD
:202AEE0082E0F09082E1E0FE9082E0E0D39E4003022B6474019082BBF0740C9082BCF0A37B
:202B0E007400F074019082BEF09082E0E09082BFF09082E0E075F002A49080B32582F582BD
:202B2E0050020583E0FAA3E0FBEA908263F0A3EBF09082E0E0908265F01219B490826612E6
:202B4E00762D9082C012764F12257D9082E0E004F06003808E009082DEE024FFB3E433FE75
:202B6E009082DEE0640224FFB3EE72E04003022BFA9082DFE09082E0F09082E1E0FE9082FB
:202B8E00E0E0D39E4003022BFA74019082BBF0740C9082BCF0A37400F074029082BEF0904F
:202BAE0082E0E09082BFF09082E0E075F002A49080F32582F58250020583E0FAA3E0FBEAEA
:202BCE00908271F0A3EBF09082E0E0908273F0121A4A90827412762D9082C012764F12251E
:202BEE007D9082E0E004F06003808E002274E39082CAF0A37482F074E59082CCF0A3748285
:202C0E00F01225EC9082E2E024FFB3E433FE9082E2E0640124FFB3EE72E04003022CA890DC
:202C2E0082E3E09082E4F09082E5E0FE9082E4E0D39E4003022CA874019082BBF0740E90E2
:202C4E0082BCF0A37400F074019082BEF09082E4E09082BFF09082E4E075F002A49080C3B1
:202C6E002582F58250020583E0FAA3E0FBEA908263F0A3EBF09082E4E0908265F01219B40D
:202C8E0090826612762D9082C012764F12257D9082E4E004F06003808E009082E2E024FF6A
:202CAE00B3E433FE9082E2E0640224FFB3EE72E04003022D3E9082E3E09082E4F09082E58C
:202CCE00E0FE9082E4E0D39E4003022D3E74019082BBF0740E9082BCF0A37400F074029092
:202CEE0082BEF09082E4E09082BFF09082E4E075F002A49081032582F58250020583E0FA38
:202D0E00A3E0FBEA908271F0A3EBF09082E4E0908273F0121A4A90827412762D9082C0126C
:202D2E00764F12257D9082E4E004F06003808E002274E79082CAF0A37482F074E99082CCC4
:202D4E00F0A37482F01225EC9082E6E024FFB3E433FE9082E6E0640124FFB3EE72E0400370
:202D6E00022DD19082E7E09082E8F09082E9E0FE9082E8E0D39E4003022DD174019082BBD9
:202D8E00F074179082BCF0A37400F074019082BEF09082E8E09082BFF09082E8E075F004D2
:202DAE00A4907FFF2582F5825002058312762D9082C012764F12257D9082E8E004F0600318
:202DCE0080A9009082E6E024FFB3E433FE9082E6E0640224FFB3EE72E04003022E4C9082D4
:202DEE00E7E09082E8F09082E9E0FE9082E8E0D39E4003022E4C74019082BBF07417908262
:202E0E00BCF0A37400F074029082BEF09082E8E09082BFF09082E8E075F004A490801F25E5
:202E2E0082F5825002058312762D9082C012764F12257D9082E8E004F0600380A9002274AF
:202E4E00EB9082CAF0A37482F074ED9082CCF0A37482F01225EC9082EAE024FFB3E433FE82
:202E6E009082EAE0640124FFB3EE72E04003022EFA9082EBE09082ECF09082EDE0FE9082C6
:202E8E00ECE0D39E4003022EFA74019082BBF0741A9082BCF0A37400F074019082BEF09030
:202EAE0082ECE09082BFF09082ECE075F002A49080D32582F58250020583E0FAA3E0FBEAEF
:202ECE00908263F0A3EBF09082ECE0908265F01219B490826612762D9082C012764F1225D0
:202EEE007D9082ECE004F06003808E009082EAE024FFB3E433FE9082EAE0640224FFB3EE37
:202F0E0072E04003022F909082EBE09082ECF09082EDE0FE9082ECE0D39E4003022F9074DE
:202F2E00019082BBF0741A9082BCF0A37400F074029082BEF09082ECE09082BFF09082EC9F
:202F4E00E075F002A49081132582F58250020583E0FAA3E0FBEA908271F0A3EBF09082EC2B
:202F6E00E0908273F0121A4A90827412762D9082C012764F12257D9082ECE004F06003802B
:202F8E008E00229082F0E075F002A49080D32582F58250020583E0C39400A3E064809480F9
:202FAE005003022FEE9082EEE0FAA3E0FB127CDE9082F0E075F002A49080D32582F582508F
:202FCE00020583E0FCA3E0FDAE02AF03ECFAEDFBEEC39AEF64806303809BB3921002304067
:202FEE009082F0E075F002A49080A32582F58250020583E0FCA3E0FD9082EEE0C39CFAA3F3
:20300E00E09DFB127CDE9082F0E075F002A49080D32582F58250020583AC02AD03E0FAA31B
:20302E00E0FB127CB9ECC39AED64806303809BB39210A21092932010030231269082F0E02B
:20304E0075F002A49081632582F58250020583E0C394FFA3E094FF40030230B0C20F120F88
:20306E00F49082F0E075F002A49081632582F58250020583C082C0839082F0E075F002A483
:20308E009081632582F58250020583E02401FAA3E03400FBEAD083D082F0A3EBF0D20F1215
:2030AE000FF474019082A7F074029082A8F0A37400F074029082AAF090804AE09082ABF0B1
:2030CE0090804BE09082ACF074009082ADF074009082AEF074009082AFF074009082B0F067
:2030EE0074009082B1F074009082B2F01224F79082F0E090804AF0742AFB7A01780290807C
:20310E0051750703127CF4200C030231269082F0E0908284F0121C4E229082F3E075F00275
:20312E00A49081132582F58250020583E0C39400A3E06480948050030231849082F1E0FA28
:20314E00A3E0FB127CDE9082F3E075F002A49081132582F58250020583E0FCA3E0FDAE025F
:20316E00AF03ECFAEDFBEEC39AEF64806303809BB392110231D69082F3E075F002A49080C3
:20318E00E32582F58250020583E0FCA3E0FD9082F1E0C39CFAA3E09DFB127CDE9082F3E042
:2031AE0075F002A49081132582F58250020583AC02AD03E0FAA3E0FB127CB9ECC39AED6443
:2031CE00806303809BB39211A21192932011030232B29082F3E075F002A49081732582F588
:2031EE008250020583E0C394FFA3E094FF400302323C9082F3E075F002A49081732582F556
:20320E008250020583C082C0839082F3E075F002A49081732582F58250020583E02401FA54
:20322E00A3E03400FBEAD083D082F0A3EBF074019082A7F074029082A8F0A37400F0740216
:20324E009082AAF090804AE09082ABF090804BE09082ACF074009082ADF074009082AEF09D
:20326E0074009082AFF074009082B0F074009082B1F074009082B2F01224F79082F3E09004
:20328E00804BF0742AFB7A017802908051750703127CF4200C030232B29082F3E0908284E5
:2032AE00F0121C4E22A212929222A21392EA22A21492972220150302337ED20B74019082D5
:2032CE00A7F074009082A8F0A37400F074049082AAF0908048E09082ABF0908049E09082D0
:2032EE00ACF0A20B74003354019082ADF0908191E09082AEF074009082AFF074009082B03F
:20330E00F074009082B1F074009082B2F01224F7D2141232BD908189E0C39400A3E0648014
:20332E0094804003023358C2131232B8908189E0FAA3E0FB127CB9EA9081AAF0A3EBF0126C
:20334E0001C7C2121232B3023375C2121232B3908189E0FAA3E0FBEA9081AAF0A3EBF01240
:20336E0001C7C2131232B87400908000F00233A7C2141232BD740090804AF0740090804BF2
:20338E00F07400908048F07400908049F0D2121232B3D2131232B8C20B229082F8E075F0BC
:2033AE0002A49080D32582F58250020583E0C39400A3E06480948050030234059082F4E058
:2033CE00FAA3E0FB127CDE9082F8E075F002A49080D32582F58250020583E0FCA3E0FDAE21
:2033EE0002AF03ECFAEDFBEEC39AEF64806303809BB392160234579082F8E075F002A49031
:20340E0080A32582F58250020583E0FCA3E0FD9082F4E0C39CFAA3E09DFB127CDE9082F857
:20342E00E075F002A49080D32582F58250020583AC02AD03E0FAA3E0FB127CB9ECC39AED85
:20344E0064806303809BB392169082F8E075F002A49081132582F58250020583E0C3940056
:20346E00A3E06480948050030234B49082F6E0FAA3E0FB127CDE9082F8E075F002A49081B4
:20348E00132582F58250020583E0FCA3E0FDAE02AF03ECFAEDFBEEC39AEF64806303809BE8
:2034AE00B392170235069082F8E075F002A49080E32582F58250020583E0FCA3E0FD908217
:2034CE00F6E0C39CFAA3E09DFB127CDE9082F8E075F002A49081132582F58250020583AC6B
:2034EE0002AD03E0FAA3E0FB127CB9ECC39AED64806303809BB392172016030235149082E0
:20350E00F8E0908048F02017030235229082F8E0908049F0A216740033FEA217EE72E04021
:20352E00030235429082F8E0908284F0121C4ED2151232C22274019082F9F09082F9E0D3D8
:20354E00940840030235919082F9E075F002A49081632582F582500205837400F0A37400D9
:20356E00F09082F9E075F002A49081732582F582500205837400F0A37400F09082F9E00481
:20358E00F080B82274019082FAF09082FAE0D3940840030235FC9082FAE075F002A490808A
:2035AE00D32582F58250020583C082C08390818FE0FAA3E0FBEAD083D082F0A3EBF09082A6
:2035CE00FAE075F002A49081132582F58250020583C082C08390818FE0FAA3E0FBEAD08322
:2035EE00D082F0A3EBF09082FAE004F0809C22A218920C2274019081D9F09082FB7CDA7D36
:20360E008175070A750600127D0212070174099081E5F09083057CE67D8175070A75060093
:20362E00127D0290830FE0FAA3E0FBEA9081F0F0A3EBF01207C922908000E0FEEE600302D3
:20364E00371D121B1E908281E0FEEE640160030236A6800908437572722043682D9036626B
:20366E007CFB7D8275070A750600127D288009084D6F64652043682B90367D7C057D8375C9
:20368E00070A750600127D28746490830FF0A37400F01236020236B4EE641060030236B7FE
:2036AE007401908000F00236CDEE642060030236D090804CE0C39401908284F0121C4E020D
:2036CE0036E5EE644060030236E890804CE02401908284F0121C4E0236FEEE640560030257
:2036EE003701A20BB392151232C27400908188F0023717EE6406600302371AA20CB3921811
:20370E001235FD7400908188F002371A023802EE64016003023805121B1E908281E0FEEE2C
:20372E006401600302377B8009084D6178202043682D9037377CFB7D8275070A75060012A9
:20374E007D288009084D6F64652043682B9037527C057D8375070A750600127D28746490F0
:20376E00830FF0A37400F0123602023789EE6410600302378C7402908000F00237A2EE6479
:20378E002060030237A590804CE0C39401908284F0121C4E0237BAEE644060030237BD90B6
:2037AE00804CE02401908284F0121C4E0237FFEE6406600302380290804CE075F002A49022
:2037CE0080C32582F582500205837400F0A37400F090804CE075F002A49081032582F582BC
:2037EE00500205837400F0A37400F07400908188F0023802023906EE6402600302390912EF
:20380E001B1E908281E0FEEE640160030238638009084D696E202043682D90381F7CFB7DF5
:20382E008275070A750600127D288009084D6F64652043682B90383A7C057D8375070A75B6
:20384E000600127D28746490830FF0A37400F0123602023871EE641060030238747403903D
:20386E008000F002388AEE6420600302388D90804CE0C39401908284F0121C4E0238A2EE0A
:20388E00644060030238A590804CE02401908284F0121C4E023903EE640660030239069007
:2038AE00804CE075F002A49080B32582F58250020583C082C08390818BE0FAA3E0FBEAD055
:2038CE0083D082F0A3EBF090804CE075F002A49080F32582F58250020583C082C0839081BF
:2038EE008BE0FAA3E0FBEAD083D082F0A3EBF07400908188F0023906023A0AEE640360039E
:20390E00023A0D121B1E908281E0FEEE640160030239678009084C696D202043682D9039A8
:20392E00237CFB7D8275070A750600127D288009084D6F64652043682B90393E7C057D8394
:20394E0075070A750600127D28746490830FF0A37400F0123602023975EE641060030239B6
:20396E00787404908000F002398EEE6420600302399190804CE0C39401908284F0121C4E49
:20398E000239A6EE644060030239A990804CE02401908284F0121C4E023A07EE64066003FE
:2039AE00023A0A90804CE075F002A49080D32582F58250020583C082C08390818FE0FAA3EF
:2039CE00E0FBEAD083D082F0A3EBF090804CE075F002A49081132582F58250020583C0825C
:2039EE00C08390818FE0FAA3E0FBEAD083D082F0A3EBF07400908188F0023A0A023AF2EE22
:203A0E0064046003023AF5121B1E908281E0FEEE64016003023A6B8009085761726E2043F7
:203A2E00682D903A277CFB7D8275070A750600127D288009084D6F64652043682B903A42AC
:203A4E007C057D8375070A750600127D28746490830FF0A37400F0123602023A79EE6410CD
:203A6E006003023A7C7400908000F0023A92EE64206003023A9590804CE0C394019082840B
:203A8E00F0121C4E023AAAEE64406003023AAD90804CE02401908284F0121C4E023AEFEE6C
:203AAE0064066003023AF290804CE075F002A49081632582F582500205837400F0A37400CF
:203ACE00F090804CE075F002A49081732582F582500205837400F0A37400F07400908188AD
:203AEE00F0023AF2023AF5227401908311F0908311E0D394084003023B8F908311E075F0D3
:203B0E0004A49081212582F58250020583C082C0831277AC00000000D083D082127840900C
:203B2E008311E075F004A49081412582F58250020583C082C0831277AC00000000D083D0CF
:203B4E0082127840908311E075F002A49080A32582F582500205837400F0A37400F09083D3
:203B6E0011E075F002A49080E32582F582500205837400F0A37400F0908311E004F0023AB1
:203B8E00FC908185E0908186F0227420FA7C017D007E047F01127B1D7B00127C05803534D1
:203BAE002D2D2D2D2D2D2D2D2D2D2D2D2D2D2D2D2D2D2D2D2D2D2D2D2D2D2D2D2D2D2D2D57
:203BCE002D2D2D2D2D2D2D2D2D2D2D2D2D2D2D2D2D2D2D2D903BAE7D007C017F347E00129D
:203BEE007B1D7B00127C05801413322A3820485620437572722E4D657465723A20127A311A
:203C0E00903BF774021279AD9000B774021279AD9000C874021279AD7D007C01E0A3FF7E31
:203C2E0002127B1D7B00127C057423FA7C017D007E047F01127B1D7E007F01908001E0FA9C
:203C4E00A3E0FB127B777B00127C0580050443414E3A903C5C7D007C017F047E00127B1D64
:203C6E007E007F01908043E0FAA3E0FB127B777420FA7C017D007E047F01127B1D7E007F58
:203C8E0001908045E0FA7B00127B777B00127C0580171650687973696B2E496E73742E2C0E
:203CAE0020556E692048443A20127A31903CA074021279AD9000C074021279AD7D007C01D5
:203CCE00E0A3FF7E02127B1D7B00127C058035342D2D2D2D2D2D2D2D2D2D2D2D2D2D2D2D63
:203CEE002D2D2D2D2D2D2D2D2D2D2D2D2D2D2D2D2D2D2D2D2D2D2D2D2D2D2D2D2D2D2D2D16
:203D0E002D2D2D2D903CDE7D007C017F347E00127B1D7B00127C05802A293F2020202020A2
:203D2E002020202020202048656C70202863206368616E6E656C3D312E2E382C20303D614C
:203D4E006C6C29903D287D007C017F297E00127B1D7B00127C05801E1D21206E202020209D
:203D6E00202020202020417474656E74696F6E204D6F64756C65903D677D007C017F1D7EF1
:203D8E0000127B1D7B00127C05801E1D23206E20202020202020202020536574204D6F6445
:203DAE00756C65205365724E72903D9A7D007C017F1D7E00127B1D7B00127C05803E3D2651
:203DCE00206E2C627228302E2E3629205365742043414E2049442C626175647261746528AD
:203DEE002832302C35302C3130302C3132352C3235302C3530302C314D487A29903DCD7DE9
:203E0E00007C017F3D7E00127B1D7B00127C05801B1A412F6120202020202020202020411E
:203E2E002052656C2E204F4E2F4F4646903E207D007C017F1A7E00127B1D7B00127C058005
:203E4E001B1A422F6220202020202020202020422052656C2E204F4E2F4F4646903E507DF7
:203E6E00007C017F1A7E00127B1D7B00127C05801D1C4320632F6320202020202020204394
:203E8E0068616E6E656C205365742F476574903E807D007C017F1C7E00127B1D7B00127CEF
:203EAE0005802A294420702C746578743C63723E20446973706C6179207465787420617438
:203ECE0020702028303D756E6C6F636B29903EB27D007C017F297E00127B1D7B00127C0582
:203EEE0080161564202020202020202020202020476574204B657973903EF17D007C017F11
:203F0E00157E00127B1D7B00127C05802221452F6520202020202020202020466F726D6177
:203F2E007420536369656E742E2F5363616C2E903F1C7D007C017F217E00127B1D7B001231
:203F4E007C05801F1E462F6620202020202020202020466174616C204C4F434B2F554E4CAB
:203F6E004F434B903F537D007C017F1E7E00127B1D7B00127C05801B1A4720632C612F67C5
:203F8E0020632C6220205368756E742F4F686D20412F42903F877D007C017F1A7E00127B97
:203FAE001D7B00127C05801A19482F6820202020202020202020416C61726D204F46462FDF
:203FCE004F4E903FB77D007C017F197E00127B1D7B00127C05801E1D4920632F6920632026
:203FEE00202020202043757272656E74732F416D7020412F42903FE67D007C017F1D7E00D5
:20400E00127B1D7B00127C05802E2D4B2F6B202020202020202020204B6579204C4F434B68
:20402E0020287374617274205761746368646F67292F554E4C4F434B9040197D007C017F25
:20404E002D7E00127B1D7B00127C058023224C20632C612F6C20632C6220204C696D6974E3
:20406E002063757272656E742073657420412F4290405C7D007C017F227E00127B1D7B0067
:20408E00127C058016154D206E2F6D20202020202020204D6F64652F6765749040947D0088
:2040AE007C017F157E00127B1D7B00127C05801A194E20632F6E2063202020202020526194
:2040CE0077206461746120412F429040BF7D007C017F197E00127B1D7B00127C05802322B3
:2040EE004F20632F6F20632020202020204C696D69742063757272656E742067657420411C
:20410E002F429040EE7D007C017F227E00127B1D7B00127C05802726702020202020202074
:20412E0020202020204C69737420616C6C205368756E74732F4F686D2028412C42299041F3
:20414E00267D007C017F267E00127B1D7B00127C058023225120632C612F7120632C62205F
:20416E002043616C6962726174652063757272656E7420412F429041627D007C017F227E49
:20418E0000127B1D7B00127C058021205220632F72206320202020202052616E6765204191
:2041AE002F4220286D696E2C6D61782990419A7D007C017F207E00127B1D7B00127C05809F
:2041CE002625532F732020202020202020202053746174757320416C61726D2F5761726EF9
:2041EE002E2028412C42299041D07D007C017F257E00127B1D7B00127C05802A2954206E39
:20420E002F74202020202020202054696D652064656C61792048562D52656C2E2028412D3D
:20422E0042292F47657490420B7D007C017F297E00127B1D7B00127C05802120552F752027
:20424E00202020202020202020556E69706F6C2E2F6269706F6C2E206D6F646590424A7DBA
:20426E00007C017F207E00127B1D7B00127C05801D1C5620632F7620202020202020204166
:20428E0076657261676520636E742F4765749042807D007C017F1C7E00127B1D7B00127CCA
:2042AE0005801A195720632F7720632020202020205761726E696E677320412F429042B2D6
:2042CE007D007C017F197E00127B1D7B00127C05801C1B582F782020202020202020202012
:2042EE004D6F6E69746F72204F4E2F4F46469042E17D007C017F1B7E00127B1D7B00127C89
:20430E0005801C1B5920632F7920632020202020205265732E2052616E676520412F429045
:20432E0043127D007C017F1B7E00127B1D7B00127C05801F1E5A20632F7A2063202020200A
:20434E0020205265732E205761726E696E677320412F429043437D007C017F1E7E00127BC4
:20436E001D7B00127C058018175E20636F646520202020202020536176652053657475709C
:20438E009043777D007C017F177E00127B1D7B00127C058035342D2D2D2D2D2D2D2D2D2D54
:2043AE002D2D2D2D2D2D2D2D2D2D2D2D2D2D2D2D2D2D2D2D2D2D2D2D2D2D2D2D2D2D2D2D4F
:2043CE002D2D2D2D2D2D2D2D2D2D9043A47D007C017F347E00127B1D7B00127C0522800110
:2043EE00009043EE7C147D8375070A750600127D287401908321F0908321E0D39408400347
:20440E0002444730980302441980F8C298E599640D600302442522908321E0908314F0906B
:20442E008321E09083142582F58250020583E599F0908321E004F080BE221243EC9083148D
:20444E00C082C08390831FD005D004127A87EC90831EF090831FE0FAA3E0FBEA908312F045
:20446E00A3EBF022908324E0FCA3E0FD8C828D83C082C083740090819AF0A37400F07408C6
:20448E0090819CF0A37400F0120146D083D082C082C08390819EE0D083D082F0908324E0AC
:2044AE00FCA3E0FD8C828D83E060030244DD908322E0FCA3E0FD8C828D837401F0908324A3
:2044CE00E0FCA3E0FD8C828D837408F00244FF908322E0FCA3E0FD8C828D83C082C08390DF
:2044EE008324E0FCA3E0FD8C828D83E0D083D082F022908094E0FEEE6401600302453090B7
:20450E00832612762D90833C7E017FFF126F0E90833C7C2C7D83750710750600127D0202C3
:20452E004618EE600302461B90832BE0640160030245AE90832612762D90832AE075F0040C
:20454E00A49080502582F5825002058312762D12750490820D12764F7406908211F0120D6F
:20456E0096127A3190821274011279AD90832AE09080942582F58250020583E0FB7A017882
:20458E0002E41279AD7441FB7A017802E41279AD7C2C7D83750710750600127D020246188E
:2045AE0090832612762D90832AE075F004A49080702582F5825002058312762D127504908D
:2045CE00820D12764F7406908211F0120D96127A3190821274011279AD90832AE090809CCE
:2045EE002582F58250020583E0FB7A017802E41279AD7441FB7A017802E41279AD7C2C7DE3
:20460E0083750710750600127D0202461B2290834CE0908228F07401908229F0120E6074EF
:20462E001F90822BF0A37400F0741F90822DF0A37400F012100F740D908241F074009082D5
:20464E0042F0A37400F0121332740D90823DF0740290823EF012125E74FB90F7D0F0740E8C
:20466E00908241F0908043E0FAA3E0FBEA908242F0A3EBF0121332740E90823DF074029074
:20468E00823EF012125E74FB90F7E0F0C20D2274019081D9F0800908536176696E672E2E7F
:2046AE009046A57CDA7D8175070A750600127D2812070174019081D8F01206B874009081A8
:2046CE00C6F0A37400F0120529908001AA82AB83EA9081C8F0A3EBF074009081CAF0A374DD
:2046EE0000F0908047AA82AB83908001AC02AD03AA82AB83ECC39AFAED9BFBEA9081CCF0C5
:20470E00A3EBF012056E74009081D8F01206B880060553617665649047207D007C017F0578
:20472E007E00127B1D7B00127C0522740190834DF090834DE0D3940840030247A490834D0F
:20474E00E075F004A4907FFF2582F5825002058312762D7B007E017FFF126F437420FA7C5D
:20476E00017D007E047F01127B1D90834DE075F004A490801F2582F5825002058312762DD8
:20478E007B007E017FFF126F437B00127C0590834DE004F0809B227E007F01908001E0FA67
:2047AE00A3E0FB127B777420FA7C017D007E047F01127B1D7E007F01908043E0FAA3E0FB8C
:2047CE00127B777420FA7C017D007E047F01127B1D7E007F01908045E0FA7B00127B777473
:2047EE0020FA7C017D007E047F01127B1D7E007F01908046E0FA7B00127B777B00127C0530
:20480E001247392274019081D8F01206B874009081D0F0A37400F0908001AA82AB83EA9087
:20482E0081D2F0A3EBF0908047AA82AB83908001AC02AD03AA82AB83ECC39AFAED9BFBEA7F
:20484E009081D4F0A3EBF012062474009081D8F01206B8908001E0FEA3E0B4FF06BEFF03B3
:20486E000248740248FB7400908001F0A37400F07400908043F0A37400F07402908045F032
:20488E00748E908046F0740190834FF090834FE0D3940840030248F890834FE075F004A476
:2048AE00907FFF2582F58250020583C082C08312759D0050C347D083D08212764F90834F03
:2048CE00E075F004A490801F2582F58250020583C082C08312759D00409C46D083D0821234
:2048EE00764F90834FE004F080A212469D22209803025A2EE59964216003024969C29812AB
:20490E004448908312E0FAA3E0FBEA908350F0A3EBF0908001E0FCA3E0FD908350E0FEA374
:20492E00E0B50507EEB5040302493D740080027401FE908350E0FAA3E0B40006BA000302F4
:20494E00495474008002740113EE72E04003024964D208024966C208025A2E200803025A96
:20496E002C7B00127B13EA90835CF090835CE0FEEE643F600302498C123B980249C7EE6438
:20498E005E60030249CA74D090819AF0A3748AF0743090819CF0A37475F012014690819EFE
:2049AE00E0FEA3E0B40406BEE0030249BE0249C412469D0249C71247A50249F9EE642360F3
:2049CE00030249FC740090819AF0A37400F0743090819CF0A37475F012014690819EE0FACA
:2049EE00A3E0FBEA908001F0A3EBF0024A55EE64266003024A58740090819AF0A37400F08C
:204A0E00741F90819CF0A37400F012014690819EE0FAA3E0FBEA908043F0A3EBF074009042
:204A2E00819AF0A37400F0740690819CF0A37400F012014690819EE0908045F0908045E0D6
:204A4E0090834CF012461C024A65EE64416003024A68D2121232B3024A75EE646160030276
:204A6E004A78C2121232B3024A85EE64426003024A88D2131232B8024A95EE646260030224
:204A8E004A98C2131232B8024AA5EE64486003024AA8C2151232C2024AB5EE646860030276
:204AAE004AB8D2151232C2024B4AEE64596003024B4D745E908322F0A37483F0745F908353
:204ACE0024F0A37483F012447290835EE090835DF090835FE0FE90835DE0D39E4003024B10
:204AEE004A90835DE075F002A49080C32582F58250020583C082C08390818DE0FAA3E0FBBD
:204B0E00EAD083D082F0A3EBF090835DE075F002A49080B32582F58250020583C082C083EF
:204B2E0090818BE0FAA3E0FBEAD083D082F0A3EBF090835DE004F06003809600024BDFEE9F
:204B4E0064796003024BE2745E908322F0A37483F0745F908324F0A37483F01244729083F8
:204B6E005EE090835DF090835FE0FE90835DE0D39E4003024BDF90835DE075F002A490819D
:204B8E00032582F58250020583C082C08390818DE0FAA3E0FBEAD083D082F0A3EBF0908381
:204BAE005DE075F002A49080F32582F58250020583C082C08390818BE0FAA3E0FBEAD083EE
:204BCE00D082F0A3EBF090835DE004F06003809600024C3EEE645A6003024C41745E90833B
:204BEE0022F0A37483F0745F908324F0A37483F012447290835EE090835DF090835FE0FEBE
:204C0E0090835DE0D39E4003024C3E90835DE075F002A49081632582F582500205837400BB
:204C2E00F0A37400F090835DE004F0600380CC00024C9DEE647A6003024CA0745E9083226D
:204C4E00F0A37483F0745F908324F0A37483F012447290835EE090835DF090835FE0FE90EF
:204C6E00835DE0D39E4003024C9D90835DE075F002A49081732582F582500205837400F08C
:204C8E00A37400F090835DE004F0600380CC00024CAEEE64456003024CB17401908094F00E
:204CAE00024CBFEE64656003024CC27400908094F0024D0AEE64536003024D0D7E007F02EB
:204CCE00908048E0FA7B00127B777E007F02908049E0FA7B00127B77A20B74003354017E3D
:204CEE00007F02FA7B00127B777E007F04908191E0FA7B00127B777B00127C05024D55EE10
:204D0E0064736003024D587E007F0290804AE0FA7B00127B777E007F0290804BE0FA7B0043
:204D2E00127B77A20B74003354017E007F02FA7B00127B777E007F04908191E0FA7B001236
:204D4E007B777B00127C05024E27EE644C6003024E2A745E908322F0A37483F0745F9083EC
:204D6E0024F0A37483F012447212019C9081A212762D90836012764F90835EE090835DF0AD
:204D8E0090835FE0FE90835DE0D39E4003024E2790835DE075F002A49080D32582F582508E
:204DAE00020583C082C08390836012762D90826A12764F90835DE090826EF01219EE908270
:204DCE006FE0FAA3E0FBEA908192F0A3EBF090818FE0FAA3E0FB127CB9EA908194F0A3EBB7
:204DEE00F090818FE0FAA3E0FBEA908196F0A3EBF01200D1D083D082C082C083908198E028
:204E0E00FAA3E0FBEAD083D082F0A3EBF090835DE004F06003024D8E00024EF9EE646C6024
:204E2E0003024EFC745E908322F0A37483F0745F908324F0A37483F012447212019C908188
:204E4E00A212762D90836012764F90835EE090835DF090835FE0FE90835DE0D39E4003029C
:204E6E004EF990835DE075F002A49081132582F58250020583C082C08390836012762D9029
:204E8E00827812764F90835DE090827CF0121A8490827DE0FAA3E0FBEA908192F0A3EBF0D3
:204EAE0090818FE0FAA3E0FB127CB9EA908194F0A3EBF090818FE0FAA3E0FBEA908196F02F
:204ECE00A3EBF01200D1D083D082C082C083908198E0FAA3E0FBEAD083D082F0A3EBF090AB
:204EEE00835DE004F06003024E6000024F9AEE644F6003024F9D745E908322F0A37483F07F
:204F0E00745F908324F0A37483F012447290835EE090835DF090835FE0FE90835DE0D39E75
:204F2E004003024F9A90835DE075F002A49080D32582F58250020583E0FAA3E0FBEA9082AB
:204F4E0063F0A3EBF090835DE0908265F01219B490826612762D90832612764F90835DE04F
:204F6E0090832AF0740190832BF012450090832C7D007C01E0A3FF7E02127B1D7B00127C0E
:204F8E000590835DE004F06003808A0002503BEE646F600302503E745E908322F0A374837B
:204FAE00F0745F908324F0A37483F012447290835EE090835DF090835FE0FE90835DE0D383
:204FCE009E400302503B90835DE075F002A49081132582F58250020583E0FAA3E0FBEA900C
:204FEE008271F0A3EBF090835DE0908273F0121A4A90827412762D90832612764F90835D4C
:20500E00E090832AF0740290832BF012450090832C7D007C01E0A3FF7E02127B1D7B001208
:20502E007C0590835DE004F06003808A000250B6EE644760030250B9745E908322F0A37413
:20504E0083F0745F908324F0A37483F012447212019C9081A212762D90836012764F90830F
:20506E005EE090835DF090835FE0FE90835DE0D39E40030250B390835DE075F004A4907FBF
:20508E00FF2582F58250020583C082C08390836012762DD083D08212764F90835DE004F09E
:2050AE00600380C2001209C8025131EE64676003025134745E908322F0A37483F0745F904F
:2050CE008324F0A37483F012447212019C9081A212762D90836012764F90835EE090835DB7
:2050EE00F090835FE0FE90835DE0D39E400302512E90835DE075F004A490801F2582F58233
:20510E0050020583C082C08390836012762DD083D08212764F90835DE004F0600380C20095
:20512E001209C802513FEE647060030251421247390251A8EE644E60030251AB745E9083BF
:20514E0022F0A37483F0745F908324F0A37483F012447290835EE090835DF090835FE0FE58
:20516E0090835DE0D39E40030251A890835DE075F002A49080A32582F582500205837E009E
:20518E007F06E0FAA3E0FB127B777B00127C0590835DE004F0600380C200025211EE646E04
:2051AE006003025214745E908322F0A37483F0745F908324F0A37483F012447290835EE0F8
:2051CE0090835DF090835FE0FE90835DE0D39E400302521190835DE075F002A49080E32535
:2051EE0082F582500205837E007F06E0FAA3E0FB127B777B00127C0590835DE004F06003BA
:20520E0080C2000252B2EE644960030252B5745E908322F0A37483F0745F908324F0A3749F
:20522E0083F012447290835EE090835DF090835FE0FE90835DE0D39E40030252B290835DAA
:20524E00E075F002A49080A32582F58250020583E0FAA3E0FBEA908263F0A3EBF090835D15
:20526E00E0908265F01219B490826612762D90832612764F90835DE090832AF074019083B8
:20528E002BF012450090832C7D007C01E0A3FF7E02127B1D7B00127C0590835DE004F060F7
:2052AE0003808A00025353EE64696003025356745E908322F0A37483F0745F908324F0A344
:2052CE007483F012447290835EE090835DF090835FE0FE90835DE0D39E4003025353908351
:2052EE005DE075F002A49080E32582F58250020583E0FAA3E0FBEA908271F0A3EBF0908327
:20530E005DE0908273F0121A4A90827412762D90832612764F90835DE090832AF074029089
:20532E00832BF012450090832C7D007C01E0A3FF7E02127B1D7B00127C0590835DE004F033
:20534E006003808A00025403EE64516003025406745E908322F0A37483F0745F908324F09C
:20536E00A37483F012447212019C9081A212762D90836012764F90835EE090835DF09083A8
:20538E005FE0FE90835DE0D39E400302540090835DE075F004A4907FFF2582F58250020588
:2053AE0083C082C08390835DE075F002A49080A32582F58250020583C082C08390836012C7
:2053CE00762DD083D082E0FAA3E0FB740112735212766012750412759D00007A44127504F3
:2053EE00D083D08212764F90835DE004F06003808D001209C80254B3EE647160030254B651
:20540E00745E908322F0A37483F0745F908324F0A37483F012447212019C9081A212762D9A
:20542E0090836012764F90835EE090835DF090835FE0FE90835DE0D39E40030254B09083F6
:20544E005DE075F004A490801F2582F58250020583C082C08390835DE075F002A49080E3FA
:20546E002582F58250020583C082C08390836012762DD083D082E0FAA3E0FB740112735230
:20548E0012766012750412759D00007A44127504D083D08212764F90835DE004F06003807B
:2054AE008D001209C80255BAEE645260030255BD745E908322F0A37483F0745F908324F0C7
:2054CE00A37483F012447290835EE090835DF090835FE0FE90835DE0D39E40030255BA90C6
:2054EE00835DE075F002A49080B32582F58250020583E0FAA3E0FBEA908263F0A3EBF09063
:20550E00835DE0908265F01219B490826612762D90832612764F90835DE090832AF0740148
:20552E0090832BF012450090832C7D007C01E0A3FF7E02127B1D7420FA7C017D007E047F6A
:20554E0001127B1D90835DE075F002A49080C32582F58250020583E0FAA3E0FBEA908263B5
:20556E00F0A3EBF090835DE0908265F01219B490826612762D90832612764F90835DE090FC
:20558E00832AF0740190832BF012450090832C7D007C01E0A3FF7E02127B1D7B00127C0573
:2055AE0090835DE004F060030254DD000256C1EE647260030256C4745E908322F0A3748316
:2055CE00F0745F908324F0A37483F012447290835EE090835DF090835FE0FE90835DE0D35D
:2055EE009E40030256C190835DE075F002A49080F32582F58250020583E0FAA3E0FBEA907B
:20560E008271F0A3EBF090835DE0908273F0121A4A90827412762D90832612764F90835D25
:20562E00E090832AF0740290832BF012450090832C7D007C01E0A3FF7E02127B1D7420FAE1
:20564E007C017D007E047F01127B1D90835DE075F002A49081032582F58250020583E0FA55
:20566E00A3E0FBEA908271F0A3EBF090835DE0908273F0121A4A90827412762D9083261202
:20568E00764F90835DE090832AF0740290832BF012450090832C7D007C01E0A3FF7E021272
:2056AE007B1D7B00127C0590835DE004F060030255E4000256EEEE645660030256F1740145
:2056CE0090819AF0A37400F074FF90819CF0A37400F012014690819EE0908185F0123AF653
:2056EE0002570CEE6476600302570F7E007F01908185E0FA7B00127B777B00127C05025750
:20570E003EEE6454600302574174D090819AF0A3748AF0743090819CF0A37475F012014614
:20572E0090819EE0FAA3E0FBEA908189F0A3EBF002575DEE647460030257607E007F01903C
:20574E008189E0FAA3E0FB127B777B00127C050257C6EE645760030257C9745E908322F083
:20576E00A37483F0745F908324F0A37483F012447290835EE090835DF090835FE0FE908331
:20578E005DE0D39E40030257C690835DE075F002A49081632582F582500205837E007F0621
:2057AE00E0FAA3E0FB127B6D7B00127C0590835DE004F0600380C20002582FEE64776003DD
:2057CE00025832745E908322F0A37483F0745F908324F0A37483F012447290835EE09083FE
:2057EE005DF090835FE0FE90835DE0D39E400302582F90835DE075F002A49081732582F5F6
:20580E0082500205837E007F06E0FAA3E0FB127B6D7B00127C0590835DE004F0600380C2D2
:20582E0000025861EE644D6003025864740090819AF0A37400F0740390819CF0A37400F0AE
:20584E0012014690819EE090835DF090835DE0908000F002587FEE646D60030258827E004D
:20586E007F01908000E0FA7B00127B777B00127C050258ACEE644360030258AF7401908196
:20588E009AF0A37400F0740890819CF0A37400F012014690819EE0908284F0121C4E025805
:2058AE00CAEE646360030258CD7E007F0190804CE0FA7B00127B777B00127C05025920EEA7
:2058CE00644460030259237B00127AAFEA908350F0A3EBF07B007C09908352127A4D7B0007
:2058EE00127C05C20A908350E09081D9F09083527CDA7D8175070A750600127D02120701B9
:20590E00908350E0FEA3E0B40006BE0003025920D20A025941EE64646003025944121AE083
:20592E007E007F0190827FE0FA7B00127B777B00127C05025951EE644B60030259541201F5
:20594E00B9D20902595EEE646B6003025961C20902596EEE64586003025971D2181235FD75
:20596E0002597EEE64786003025981C2181235FD025992EE64556003025995748E908046DA
:20598E00F01209C80259A6EE647560030259A97486908046F01209C8025A00EE642A600399
:2059AE00025A037B00127B13EA90835CF090835CE0FEEE644360030259CDD20D0259D7EEAA
:2059CE00646360030259DAC20D025A007407FA7C017D007E047F01127B1D800302203F90A0
:2059EE0059EB7D007C017F027E00127B1D7B00127C05025A297407FA7C017D007E047F01AE
:205A0E00127B1D800302203F905A147D007C017F027E00127B1D7B00127C05025A2EC29857
:205A2E0022908001E0FAA3E0FB9083647F07E4126F23908043E0FAA3E0FB90836E7F05E4B4
:205A4E00126F237423FB7A01127A317802E41279AD90836474011279AD7CFB7D8275070A14
:205A6E00750600127D0280040343414E127A31905A7674021279AD90836E74011279AD7C3E
:205A8E00057D8375070A750600127D0274D090830FF0A37407F012360222908186E0C394C3
:205AAE0001908186F07401908378F0908378E0D394084003025E7E908378E0908207F0747D
:205ACE0079908208F0A37483F0747B90820AF0A37483F0120B34908379E0FAA3E0FBEA9077
:205AEE0082EEF0A3EBF0908378E09082F0F0122F9190837BE0FAA3E0FBEA9082F1F0A3EB3A
:205B0E00F0908378E09082F3F0123127908378E075F004A49081212582F58250020583C05B
:205B2E0082C083908378E075F004A49081212582F5825002058312782A908379E0FAA3E053
:205B4E00FBE41277C6127723D083D082127840908378E075F004A49081412582F5825002B4
:205B6E000583C082C083908378E075F004A49081412582F5825002058312782A90837BE026
:205B8E00FAA3E0FBE41277C6127723D083D082127840908186E0D394004003025E75300B00
:205BAE0003025E2B908378E075F004A49081212582F5825002058312782A74021277C6909E
:205BCE008185E0FA7B007401127352127504127331EA908379F0A3EBF0908378E075F00417
:205BEE00A49081412582F5825002058312782A74021277C6908185E0FA7B007401127352F9
:205C0E00127504127331EA90837BF0A3EBF0908379E0FAA3E0FBEA9082F4F0A3EBF09083FA
:205C2E007BE0FAA3E0FBEA9082F6F0A3EBF0908378E09082F8F01233A8908378E075F002FF
:205C4E00A49080C32582F58250020583E0FCA3E0FDECFAEDFB908379E0D39AA3E0648063FA
:205C6E0003809B5003025CAAC004C00574799082CEF0A37483F0908378E075F002A4908047
:205C8E00C32582F58250020583AA82AB83EA9082D0F0A3EBF0122642D005D004908378E019
:205CAE0075F002A49080B32582F58250020583E0FCA3E0FDECFAEDFB908379E0C39AA3E09A
:205CCE0064806303809B4003025D0DC004C00574799082CEF0A37483F0908378E075F00200
:205CEE00A49080B32582F58250020583AA82AB83EA9082D0F0A3EBF0122642D005D00490F0
:205D0E008378E075F002A49081032582F58250020583E0FCA3E0FDECFAEDFB90837BE0D318
:205D2E009AA3E064806303809B5003025D70C004C005747B9082CEF0A37483F0908378E074
:205D4E0075F002A49081032582F58250020583AA82AB83EA9082D0F0A3EBF0122642D0053B
:205D6E00D004908378E075F002A49080F32582F58250020583E0FCA3E0FDECFAEDFB908393
:205D8E007BE0C39AA3E064806303809B4003025DD3C004C005747B9082CEF0A37483F0907E
:205DAE008378E075F002A49080F32582F58250020583AA82AB83EA9082D0F0A3EBF0122628
:205DCE0042D005D00474799082CEF0A37483F0908378E075F002A49080A32582F5825002EA
:205DEE000583AA82AB83EA9082D0F0A3EBF0122642747B9082CEF0A37483F0908378E075D6
:205E0E00F002A49080E32582F58250020583AA82AB83EA9082D0F0A3EBF01226429083785A
:205E2E00E075F004A49081212582F58250020583C082C0831277AC00000000D083D08212CC
:205E4E007840908378E075F004A49081412582F58250020583C082C0831277AC0000000000
:205E6E00D083D082127840908378E004F0025AB9908186E0D394004003025E92908185E0A8
:205E8E00908186F02290837DE0D394085003025EA5740890837DF07401908394F090837D7C
:205EAE00E0FE908394E0D39E4003025EF7908394E090838A2582F58250020583C082C083C3
:205ECE0090837EE0FCA3E0FD8C828D83E0D083D082F090837EE004F07004A3E004F09083D1
:205EEE0094E004F0600380B50090837DE090838AF090838A7C807D8375070A750600127D6E
:205F0E00022280080743414E2049443A905F137D007C017F077E00127B1D7E007F05908348
:205F2E0095E0FAA3E0FB127B6D80040320443A905F3A7D007C017F037E00127B1D908397D0
:205F4E00E0D394005003025F9B740190839AF0908397E0FE90839AE0D39E4003025F9B9036
:205F6E008398E0FCA3E0FD8C828D837E007F04E0FA7B00127B77908398E004F07004A3E0AE
:205F8E0004F090839AE004F0600380C3007B00127C052290839BE090839FF0A3740000F071
:205FAE007C087D0090839FE0FAA3E0FB127CC490839CE0FC7D00EA4CFAEB4DFBEA90839D71
:205FCE00F0A3EBF0229083A1E090825DF09083A2E0FAA3E0FBEA908293F0A3EBF012249858
:205FEE00908295E0FAA3E0FBEA90825EF0A3EBF09083A4E0908260F09083A5AA82AB83EAD7
:20600E00908261F0A3EBF0121928221201BC9083AEE0908249F01214E990824A12782A74CE
:20602E00011277C6EA9083AFF0A3EBF09083AEE0908257F074B9908258F0A37483F09083CA
:20604E00B1AA82AB83EA90825AF0A3EBF01217B4200D0302608E9083AFE0FAA3E0FBEA90D2
:20606E008395F0A3EBF09083B9E0908397F09083B1AA82AB83EA908398F0A3EBF0125F10A4
:20608E009083AFE0FAA3E0FBEA908290F0A3EBF0122483908292E0FEEE6003026103740177
:2060AE009082A7F074009082A8F0A37400F074049082AAF0908048E09082ABF0908049E0C2
:2060CE009082ACF0A20B74003354019082ADF0908191E09082AEF074009082AFF074009051
:2060EE0082B0F074009082B1F074009082B2F01224F7026119EE6401600302611C9083B17F
:20610E00E0640124FFB392151232C2026171EE6402600302617474019082A7F074029082A1
:20612E00A8F0A37400F074029082AAF090804AE09082ABF090804BE09082ACF0740090823A
:20614E00ADF074009082AEF074009082AFF074009082B0F074009082B1F074009082B2F0D6
:20616E001224F702618FEE640460030261929083B1E09082D2F09083B2E09082D3F012261A
:20618E0077026261EE6405600302626474B29082CAF0A37483F074BA9082CCF0A37483F031
:2061AE001225EC9083B1E024FFB3E433FE9083B1E0640124FFB3EE72E0400302620990833D
:2061CE00B2E09083B9F09083BAE0FE9083B9E0D39E40030262099083B9E075F002A4908123
:2061EE00632582F582500205837400F0A37400F09083B9E004F0600380CC009083B1E024B4
:20620E00FFB3E433FE9083B1E0640224FFB3EE72E040030262619083B2E09083B9F090830D
:20622E00BAE0FE9083B9E0D39E40030262619083B9E075F002A49081732582F582500205E3
:20624E00837400F0A37400F09083B9E004F0600380CC000262A0EE640660030262A390831A
:20626E00B1E0C3940240030262869083B1E0640124FFB392121232B39083B2E0C394024041
:20628E00030262A09083B2E0640124FFB392131232B80262FAEE640760030262FD740190E8
:2062AE0082A7F074079082A8F0A37400F074029082AAF0A2927400339082ABF0A2EA7400E1
:2062CE00339082ACF074009082ADF074009082AEF074009082AFF074009082B0F074009039
:2062EE0082B1F074009082B2F01224F7026318EE6409600302631B9083B1E09082D6F09051
:20630E0083B2E09082D7F01227F5026336EE640B60030263399083B1E09082DAF09083B215
:20632E00E09082DBF0122939026354EE640D60030263579083B1E09082DEF09083B2E0902E
:20634E0082DFF0122AB7026372EE640F60030263759083B1E09082E2F09083B2E09082E354
:20636E00F0122BFB0263A0EE641160030263A39083B1E090839BF09083B2E090839CF0127C
:20638E005FA190839DE0FAA3E0FBEA908189F0A3EBF00263F8EE641360030263FB7401906B
:2063AE0082A7F074129082A8F0A37400F074029082AAF090818AE09082ABF0908189E0902B
:2063CE0082ACF074009082ADF074009082AEF074009082AFF074009082B0F074009082B1C8
:2063EE00F074009082B2F01224F702641DEE641460030264209083B1E0640160030264178F
:20640E00748E908046F002641D7486908046F0026521EE6416600302652474B29082CAF093
:20642E00A37483F074BA9082CCF0A37483F01225EC9083B312762D90829712764F1224BE2C
:20644E0090829B12762D9083B312764F9083B1E024FFB3E433FE9083B1E0640124FFB3EED3
:20646E0072E040030264BC9083B2E09083B9F09083BAE0FE9083B9E0D39E40030264BC9039
:20648E0083B9E075F004A4907FFF2582F58250020583C082C0839083B312762DD083D0821A
:2064AE0012764F9083B9E004F0600380C2009083B1E024FFB3E433FE9083B1E0640224FFF6
:2064CE00B3EE72E0400302651E9083B2E09083B9F09083BAE0FE9083B9E0D39E4003026520
:2064EE001E9083B9E075F004A490801F2582F58250020583C082C0839083B312762DD0833D
:20650E00D08212764F9083B9E004F0600380C2001209C802653FEE641860030265429083ED
:20652E00B1E09082E6F09083B2E09082E7F0122D3F0266F4EE641960030266F774B2908207
:20654E00CAF0A37483F074BA9082CCF0A37483F01225EC9083B312762D90829712764F1233
:20656E0024BE90829B12762D9083B312764F9083B1E024FFB3E433FE9083B1E0640124FF71
:20658E00B3EE72E040030266389083B2E09083B9F09083BAE0FE9083B9E0D39E4003026643
:2065AE00389083B9E075F002A49080D32582F58250020583C082C0839083B312762D9082F1
:2065CE006A12764F9083B9E090826EF01219EE90826FE0FAA3E0FBEA908192F0A3EBF090D3
:2065EE00818FE0FAA3E0FB127CB9EA908194F0A3EBF090818FE0FAA3E0FBEA908196F0A3C5
:20660E00EBF01200D1D083D082C082C083908198E0FAA3E0FBEAD083D082F0A3EBF0908373
:20662E00B9E004F0600302659F009083B1E024FFB3E433FE9083B1E0640224FFB3EE72E0A7
:20664E0040030266F49083B2E09083B9F09083BAE0FE9083B9E0D39E40030266F49083B9F9
:20666E00E075F002A49081132582F58250020583C082C0839083B312762D90827812764FA4
:20668E009083B9E090827CF0121A8490827DE0FAA3E0FBEA908192F0A3EBF090818FE0FAB6
:2066AE00A3E0FB127CB9EA908194F0A3EBF090818FE0FAA3E0FBEA908196F0A3EBF0120001
:2066CE00D1D083D082C082C083908198E0FAA3E0FBEAD083D082F0A3EBF09083B9E004F013
:2066EE00600302665B00026712EE641B60030267159083B1E09082EAF09083B2E09082EB6B
:20670E00F0122E4D026728EE641E600302672B9083B1E0908185F0123AF602677EEE641F32
:20672E00600302678174019082A7F0741F9082A8F0A37400F074019082AAF0908185E09075
:20674E0082ABF074009082ACF074009082ADF074009082AEF074009082AFF074009082B04A
:20676E00F074009082B1F074009082B2F01224F70268BCEE643160030268BF74B29082CA68
:20678E00F0A37483F074BA9082CCF0A37483F01225EC9083B1E024FFB3E433FE9083B1E095
:2067AE00640124FFB3EE72E0400302682E9083B2E09083B9F09083BAE0FE9083B9E0D39E4C
:2067CE00400302682E9083B9E075F002A49080C32582F58250020583C082C08390818DE04B
:2067EE00FAA3E0FBEAD083D082F0A3EBF09083B9E075F002A49080B32582F58250020583A4
:20680E00C082C08390818BE0FAA3E0FBEAD083D082F0A3EBF09083B9E004F06003809600DB
:20682E009083B1E024FFB3E433FE9083B1E0640224FFB3EE72E040030268BC9083B2E090FD
:20684E0083B9F09083BAE0FE9083B9E0D39E40030268BC9083B9E075F002A490810325825B
:20686E00F58250020583C082C08390818DE0FAA3E0FBEAD083D082F0A3EBF09083B9E07520
:20688E00F002A49080F32582F58250020583C082C08390818BE0FAA3E0FBEAD083D082F061
:2068AE00A3EBF09083B9E004F060038096000268F6EE643360030268F99083B1E090819241
:2068CE00F0A3740000F07401908194F0A37400F07408908196F0A37400F01200D1908198FC
:2068EE00E0908284F0121C4E02694CEE6434600302694F74019082A7F074349082A8F0A33B
:20690E007400F074019082AAF090804CE09082ABF074009082ACF074009082ADF0740090B2
:20692E0082AEF074009082AFF074009082B0F074009082B1F074009082B2F01224F70269F7
:20694E009CEE6435600302699FC20A9083B1E09081D9F09083B9E0C3940190837DF09083B8
:20696E00B2AA82AB83EA90837EF0A3EBF0125E939083807CDA7D8175070A750600127D0298
:20698E001207019083B1E0700302699CD20A0269F5EE643660030269F874019082A7F07495
:2069AE00369082A8F0A37400F074019082AAF0121AE090827FE09082ABF074009082ACF075
:2069CE0074009082ADF074009082AEF074009082AFF074009082B0F074009082B1F074007C
:2069EE009082B2F01224F7026A42EE64376003026A459083B1E0FEEE6003026A10C2090221
:206A0E006A1AEE64016003026A1DD209026A28EE64026003026A2B1201B9026A3FEE64031C
:206A2E006003026A421201B9D2BE8003026A3F80F9026A42026A81EE64386003026A84902C
:206A4E0083B1E0908192F0A3740000F07400908194F0A37400F07404908196F0A37400F054
:206A6E001200D1908198E09083B9F09083B9E0908000F0026AD7EE64396003026ADA740148
:206A8E009082A7F074399082A8F0A37400F074019082AAF0908000E09082ABF0740090829D
:206AAE00ACF074009082ADF074009082AEF074009082AFF074009082B0F074009082B1F073
:206ACE0074009082B2F01224F7026B33EE643A6003026B3674019082A7F0743A9082A8F0AB
:206AEE00A37400F074069082AAF074019082ABF074539082ACF0908002E09082ADF0908013
:206B0E0001E09082AEF0908044E09082AFF0908043E09082B0F074009082B1F0740090825F
:206B2E00B2F01224F7026BDDEE643B6003026BE09083B1E090839BF09083B2E090839CF06B
:206B4E00125FA190839DE0FEA3E0B40106BE5303026B65740080027401FEC0069083B3E08E
:206B6E0090839BF09083B4E090839CF0125FA1D006908001E0FCA3E0FD90839DE0FAA3E0C1
:206B8E00B50507EAB50403026B9C74008002740113EE82E04003026BDD9083B5E090839BC6
:206BAE00F09083B6E090839CF0125FA190839DE0FAA3E0FBEA908043F0A3EBF09083B7E020
:206BCE00908045F0908045E090834CF012461C026C0BEE643C6003026C0E74019083A1F06B
:206BEE00743C9083A2F0A37400F09000B77CA47D8375070A750600127D28125FD3026C3921
:206C0E00EE643D6003026C3C74019083A1F0743D9083A2F0A37400F09000C87CA47D837567
:206C2E00070A750600127D28125FD3026C95EE643E6003026C9874019082A7F0743E9082E1
:206C4E00A8F0A37400F074019082AAF0908227E09082ABF074009082ACF074009082ADF05B
:206C6E0074009082AEF074009082AFF074009082B0F074009082B1F074009082B2F0122412
:206C8E00F77400908227F0026C989083AEE075F010A490F7002582F5825002058374FDF0B2
:206CAE0022300B03026CC030EB03026CC0D2151232C222C0D075D000C0E0C0F0C082C08333
:206CCE009083BB127D7A90F702E0C394029083AEF01260199083BB127D9DD083D082D0F072
:206CEE00D0E0D0D03274009081D8F01206B8758680E5A9FEEE544064406003026D1B9081BC
:206D0E0091E02401908191F0D20E026D237400908191F0C20E7B00127EE1758DF575900FFE
:206D2E0075E8FFD2B3D2B57400908000F0121C3F1209A99000B77CFB7D8275070A7506007A
:206D4E00127D289000C87C057D8375070A750600127D2874D090830FF0A37407F01236022F
:206D6E00124812125A2F908045E090834CF012461C1209C8800908202020202043682D908A
:206D8E006D847CFB7D8275070A750600127D288009084D6F64652043682B906D9F7C057D20
:206DAE008375070A750600127D2874D090830FF0A37407F01236027401908185F0740090DD
:206DCE008189F0A37400F0123AF61235921235431223C77401908284F0121C4EC21812356B
:206DEE00FDC20DD2087400908094F0C2151232C2D2151232C21201BC125AA8126CAF121CCF
:206E0E00911201BC1236451248FC80E980FE885D8B5C8C5E7524017A007B00127352C21A42
:206E2E00752500127DD0C219EAC3942D700BD219752402127DD0026E53EAC3942B70067588
:206E4E002402127DD0EAC39430B333FBEAC394396001B3B3EB82E033FBEAC3942EC37001EE
:206E6E00D3EB72E04003026EAE201A03026E7F0525EAC3942E6003026E8DD21A026EA9C0A9
:206E8E00027A0A7B00127352127486D0E0C39430FA7B001273521274120524127DD080A538
:206EAE00201A03026ECFE525C394006001B34003026ECF7A0A7B0012735212750415258036
:206ECE00E5201903026ED812731F22ECC0E0E604FCF531087B05126E1CD00112761C127AB8
:206EEE00A822C083C0828C828D83E0A304FCF5317B06126E1CD082D08312764F127AA8227F
:206F0E00C082C083A37B06755E00126F43E55ED083D082F022C082C083A37E06755E00604A
:206F2E0005127B6D8003127B77E55ED083D082F022127E5A228B5C8E448F26792712761C05
:206F4E00752C0778271275E17A007B001273521276714003026F77D21B78271275E112730B
:206F6E001F792712761C026F79C21B78271275E17A007B0012735212767170030271CB78E4
:206F8E00271275E1C082C08312759D8096184BD083D0821276715003026FC178271275E108
:206FAE007A0A7B00127352127504792712761C052C80CC78271275E1C082C08312759DFFF2
:206FCE00237449D083D08212767133FA7407C3952CC39526C36001D33313EA82E0400302AD
:206FEE00700878271275E17A0A7B00127352127486792712761C152C80B978271275E1C09D
:20700E0082C08312759D0000003FD083D0821274121273DB12724EE526C394FFC37001D363
:20702E0033FAE52CC394076001B3EA72E040030270FCE52CC3947F6001B3335401240CFAF8
:20704E00A21B3354012AF545E52CFA7B00127B18127CDE7C097D00C3127D646001B34003D3
:20706E000270730545E52CFA7B00127B18127CDE7C637D00C3127D646001B34003027090D1
:20708E000545854545E544C3954550030270AC7420FA126F3F0545E545600380E800201B8A
:2070AE00030270B8742DFA126F3F7430FA126F3F742EFA126F3F7545037409C39545500356
:2070CE000270E4E545243AF8E6FA126F3F0545E545600380E4007445FA126F3FE52CFA7BF8
:2070EE0000127B18AE5C7F01127B770271C8754500E545243AF8E6C39420C37001D333FC47
:20710E007409C39526FDE545C39DEC82E04003027124054580DB201B0302712C1545740C5B
:20712E00C39545F545E544C39545500302714C7420FA126F3F0545E545600380E800201BCA
:20714E0003027158742DFA126F3FE52C2526C394076001B34003027170E52C2402F52B02AB
:20716E0071777409C39526F52B7545027409C3954550030271C8E545243AF8E6C39420704D
:20718E000302719FE545243AF8E6FA126F3F0271AFE545C3952B50030271AF7430FA126F49
:2071AE003FE545C3952B60030271BF742EFA126F3F0545E545600380B30002724DE526C34B
:2071CE0094FF6003027206754504E544C3954550030271F17420FA126F3F0545E5456003D1
:2071EE0080E8007430FA126F3F742EFA126F3F7430FA126F3F02724D74032526F545E5441B
:20720E00C3954550030272257420FA126F3F0545E545600380E8007430FA126F3F742EFA50
:20722E00126F3F754501E526C39545500302724D7430FA126F3F0545E545600380E800224A
:20724E00792D12781F800B0A20202020202020202030C082C083907256793A75070A127D47
:20726E001FD083D082754509782D12780E7A007B0074001277C612784B6001B340030272E4
:20728E00CCE545243AF8C000782D12780E7A0A7B0074001277C612779574011277C6D00023
:2072AE00EA2430F61545782D12780E7A0A7B0074001277C6127788792D12781F80AA22E5A2
:2072CE0058A2E7921CD2E7F558E553A2E7921DD2E7F553E559C395544011E5596554601CEC
:2072EE00C3785012788505540272E8E5546559600BC3785512788505590272F922E6C39703
:20730E00F60809E697F60809E697F60809E697F622E5596006E558B2E7F55822E558C2E7EC
:20732E00F55822E55820E70E12759D0000003F1274121273B72212759D0000003F12740F2D
:20734E001273B72260201279018B588A57755600755500EBA2E7921C500578551278D77542
:20736E00598E127898221279018B588A57755600755500C21C80E8E558A2E7921CD2E7F587
:20738E0058C3E559949EF559500FE559601A7855C31278850559027398E559600B7855C3AC
:2073AE0012787515590273A722E5596018127385AA55AB56301C0AEAF42401FAEBF43400EE
:2073CE00FB1278EF227A007B001278EF22E5596023127385301C1CE555F42401F555E5566E
:2073EE00F43400F556E557F43400F557E558F43400F558227555007556007557007558005A
:20740E002212731FE559603CE55460351272CDA21C92E7A21D65D020E7137950785512783A
:20742E00C450077855127885055902744B7950785512730B500778551278D7B21C1278988D
:20744E00221276601278EF22E687F0A4FCADF008E687F0A42DFDE435F0FEE433FF1809E688
:20746E0087F0A42DFDE5F03EFEE43FFF08E687F0A42EFEEF35F0FF22E559700302744FE5C1
:20748E00547003027452E553A2E7921CD2E7F553E558A2E7D2E7F5585002B21C785779505B
:2074AE00127456EEFAEFFB78557952127456EE2AFAEF3BFB921D78577952127456EC2AF535
:2074CE0055ED3BF556E43EC0D0A21D3400F557E4D0D03FF558E55425592482F55912789808
:2074EE002275547F7553FF7552FF7551FF7550FF1278EFD2D222E55960E7E5547003027418
:20750E0052E553A2E7921CD2E7F553E558A2E7D2E7F5585002B21CC37850127885C3785585
:20752E00127885AC50AD51AE52AF5375500075510075520075530075F02015F0E5F0603524
:20754E00C3EC9555ED9556EE9557EF95584011C3EC9555FCED9556FDEE9557FEEF9558FF88
:20756E00B37850127875E5D0541804040404F812787502754850057850127885E554C2D79E
:20758E0095592480F5541278EF127898C2D222127901D083D08278557600087904740093B1
:2075AE00F608A319E970F6C082C0831275C12212790122E558A2E7E55933F559E55892E7DC
:2075CE00F55822E558A2E7E55913F559E55892E7F55822E8C0E0127901D0E0F879557700A3
:2075EE00097F04127CED1275C122E55530E71E7855E62401F608E63400F608E63400F60897
:20760E00E63400F6500778551278850559221275F81275D178567F04127CED1278EF221249
:20762E00790179557700097F04127CFB1275C12212790179557700097F04127D1F1275C1AB
:20764E00221275F81275D178567F04127CF41278EF22785579507A05E6FBE7F6EBF70809EF
:20766E00DAF622E553A2E7B3E55413F554E55392E7F553E558A2E7B3E55913F559E5589221
:20768E00E7F558E55920E70DE55420E708785479597F058006785979547F05C3E796700490
:2076AE001819DFF7FA13FB127980127980EB33EA221275BD12748622E55833921C50031278
:2076CE007700E55333921D5019C374009550F55074009551F55174009552F55274009553A3
:2076EE00F55322A21C33F8A21D336830E0F412770022C374009555F55574009556F5567497
:20770E00009557F55774009558F55822E55830E70312770022785579501278C4227850790A
:20772E0055C37A04E697F70809DAF922785079557A04E657F70809DAF922785079557A04C9
:20774E00E647F70809DAF922E55560097850127885155580F31278EF22E555600978501282
:20776E007875155580F31278EF221276C6127913C378551278851276F1221276C612793C5B
:20778E001278EF1276F1221276C612793C8C508D518E528F5378501278851278EF22127939
:2077AE0001D083D08278557904740093F608A319E970F6C082C08322600814602714602C71
:2077CE0080191279018A558B56EB30E7077557FF7558FF22755700755800221279018A55CE
:2077EE008B5680F0AA55AB561278EF2275599EE558A2E7921C500578551278D712789822E8
:20780E00E8C0E0127901D0E0F879557F04127CED2278557F04127CED1278EF221279017945
:20782E00557F04127CFB2212790179557F04127D1F2278557F04127CF41278EF22E55864FC
:20784E0080F8C3E5536480987010E5529557700AE55195567004E5509555FBACD0127980D8
:20786E001279808CD0EB22E633F608E633F608E633F608E633F622080808E613F618E613F8
:20788E00F618E613F618E613F6227920E55820E71C7855C3127875155919E970EF7559008F
:2078AE0075580075570075560075550022E558A21C92E7F55822E627F60809E637F608094F
:2078CE00E637F60809E637F622E6F42401F608E6F43400F608E6F43400F608E6F43400F628
:2078EE00227859795475F005E7F6181915F0E5F070F6227850795575F005E7F6080915F0ED
:20790E00E5F070F6227C007D007E007F0075F02115F0E5F06017785512788530D7077804C9
:20792E0079501278C4780412788502791E227C007D007E007F0075F021C3EC9555ED9556EF
:20794E00EE9557EF95584011C3EC9555FCED9556FDEE9557FEEF9558FFB37850127875E596
:20796E00D0541804040404F812787515F0E5F070C8221278EF22D046D047C050C051C05287
:20798E00C053C054C047C04622D046D047D054D053D052D051D050C047C04622027A106091
:2079AE00FB1460317400936025F54AA3740093858246858347054B854882854983F0A38500
:2079CE008248858349854682854783D54ADD9083DAE54BF022E06023F54AA3E085824685C0
:2079EE008347054B854882854983F0A3858248858349854682854783D54ADF9083DAE54BD5
:207A0E00F022E66011F54A854882854983054B08E6F0A3D54AF78582488583499083DAE5B7
:207A2E004BF0228582468583479083DA7400F0F54BA385824885834985468285478322AD00
:207A4E0082AE837F008B5C127DD0EA640D6006A30FEAF0DCF28D828E83EFF022ECC0E07B5D
:207A6E0005E608885D04F55EF531127AAFD0E0F8EAF608EBF6127AA822C082C0838C828D81
:207A8E00837B06E0A304F55EF531127AAFD083D082EAF0A3EBF0127AA822C3E531955EFC7E
:207AAE00228B5C753400753500127DD08A36C200E536642D7007D200127DD08A36E536C389
:207ACE009430B333FAE536C394396001B3B3EA82E0501F7C0A7D00AA34AB35127C1AE53643
:207AEE00C394302AF534EB3400F535127DD08A3680CB30000BAA34AB35127CB98A348B352D
:207B0E00AA34AB35228B5C027DD030E7011B228D5CECC39F400E600CFCEAFD7A20127E5A94
:207B2E00DCF9EDFAEF600FEE602A14601514601B146004127E5A22EAFA127E5AEBFA127EC6
:207B4E005A22E6FA127E5A08DFF822E0A3FA127E5ADFF822740093A3FA127E5ADFF6228E5D
:207B6E005C8F448A378B3880218E5C8F448A378B38EB30E715D21BE54460021544AA37ABEE
:207B8E0038127CB98A378B388002C21B754504E545243AF87C0A7D00AA37AB38127C4CEAAC
:207BAE002430F67C0A7D00AA37AB38127C3C8A378B38E544600215441545E537453870CF42
:207BCE00753901E544C39539400B7A20127E5A0539E53970EE301B057A2D127E5A05457406
:207BEE0004C395454010E545243AF8E6FA127E5A0545E54570E9228B5C7A0D127E5A7A0A71
:207C0E00127E5A2222EA2CFAEB3DFB22EEC0E0EFC0E0EA8CF0A4FEAFF0EA8DF0A42FFFEBEB
:207C2E008CF0A42FFBEEFAD0E0FFD0E0FE22EEC0E0EFC0E0127C70D0E0FFD0E0FE22BB0030
:207C4E000ABD0007EA8CF084AAF022EEC0E0EFC0E0127C70C3EF13FBEE13FAD0E0FFD0E06D
:207C6E00FE22BB000DBD000AEA8CF084FAAEF07F0022E8C0E0E9C0E075F0117E007F00EEB2
:207C8E00F8EFF9C2D7EE9CFEEF9DFFB34004E8FEE9FFEA33FAEB33FBEE33FEEF33FF15F010
:207CAE00E5F070DBD0E0F9D0E0F822EBF4FBEAF404FA70010B22EC6009C3EA33FAEB33FB87
:207CCE00DCF722EC6009C3EB13FBEA13FADCF722EB30E70AEAF42401FAEBF43400FB22E685
:207CEE00F70809DFFA22E6F008A3DFFA22E0F709A3DFFA22EF60010EE0A3AA82AB838C8230
:207D0E008D83F0A3AC82AD838A828B83DFEADEE822740093F709A3DFF822EF60010E740014
:207D2E0093A3AA82AB838C828D83F0A3AC82AD838A828B83DFE8DEE622E6FCE0FDEC600EB6
:207D4E00ED601008A31C1DC3E09660F1B322ED6003D322ECC322EA9CEDF5F06480FDEB64D7
:207D6E00809DADF022E608F0A3D9FA22E8F0A3E9F0A378027906127D7378467914127D7364
:207D8E00A21C33A21D33F022E0A3F608D9FA22E0C0E0A3E0C0E0A378027906127D96784648
:207DAE007914127D96E013921D13921CD001D000228A828B8374007390842B85825A858334
:207DCE005B22E55C60491414605514607D14607B14602F14601F14601030C0FDC2C0E5C1A2
:207DEE00FA940D6003127E5A22E59B30E0FBC2E0F59BAA9C22155EE55E6004E0A3FA227A13
:207E0E000D22155EE55E60F7A85DE6055DFA223098FDC298E599FA940D6003127E5A22D236
:207E2E00AF20B2FBC2AF7DBADDFE20B2F27A07C3127E53127E5313A2B2DAF513C313127EB8
:207E4E0053FAD2AF227DBADDFE222222E55C603914603F14605214607814607614602114DA
:207E6E00601814600930C1FDEAF5C1C2C122E59B30E1FBC2E1F59B8A9C22EAF0A3055E22C3
:207E8E00EAA85DF6055D055E223099FDEAF599C29922C083C082906100E0E020E7FB906223
:207EAE0000EAF0D082D08322C2AFC2B5127EDA127EDA7C07EA13FA92B5127EDA127EDADCE6
:207ECE00F3D2B5127EDA127EDAD2AF227DBADDFE222222EB602AB40708759DDC759B9380E2
:207EEE001EB4081BE589540F2420F589C2C7D2C6758DFAD28EE5874480F587D2C4D2C12278
:207F0E00E589540F2420F589C29FD29E758DFAD28EE5874480F587D29CD299C20122755F55
:1E7F2E0080D000D001855F81C001C00022755F60D000D001855F81C001C000D21E223F
:00000001FF
